:020000020000FC
:100000000C9405010C9430000C9431000C943200D7
:100010000C9433000C9434000C9435000C9436008E
:100020000C9437000C9441000C94A9000C94AA0085
:100030000C94AB000C94AC000C94AD000C94AE008E
:100040000C94B8000C94B9000C94BA000C94EE0017
:100050000C94EF000C94F0000C9403010C94040138
:1000600018951895189518951895189518950F9333
:100070000FB70F93A9B26894F7F80F910FBF0F91C4
:1000800018950F930FB70F930F92EF93FF93059966
:1000900009C00093BA000091B200689400F900937F
:1000A000B20010C00091B20000FF0CC06894F5F8D7
:1000B000E89400F90093B20008E00093A10008E57D
:1000C0000093A0000091AB0000FF04C0009163000A
:1000D000039503C0009163000A95077000936300C5
:1000E0001A95000011F40C9488000CEFE02F0BE03F
:1000F000F02F00916300E00F00E0F01FC895002D85
:100100000F70002E05B3007F000E05BA0C948A0014
:1001100000E005BD0E945906F5FE14C00091A10043
:100120000A9521F408E00093A10003C00093A10008
:1001300009C00091A0000A9519F4E894F5F802C0EE
:100140000093A000FF91EF910F900F910FBF0F91BF
:100150001895189518951895189518950F930FB729
:100160000F9308E003BF95980F910FBF0F9118955B
:10017000189518950F930FB70F93AF93BF93F7FE92
:1001800024C0919AF1FC0FC000E00093A60000E0AB
:100190000093AD0003E00093AE0000E00093A400E4
:1001A00003E00093A5006894F1F8A091A400B09139
:1001B000A5000CB10D93A093A400B093A5000091ED
:1001C000A60003950093A60001C0ACB06894F7F8B0
:1001D000BF91AF910F910FBF0F911895189518957A
:1001E0000093B5000FB70093B60004B100939C00D4
:1001F00005B100939D0000E007B90091B6000FBF64
:100200000091B5001895189518950EEF0DBF0FE0E9
:100210000EBF0FEF0BBB07EF07BB0FE608BB00EFEE
:1002200005BB0BEF01BB0FED02BB00E002B90FEF06
:1002300003B900E6E02F00E0F02F00E0002E0E945E
:10024000D60508E90AB90FE509B900E007B900E0E9
:1002500000936B0002E000936C0000E000936D00DF
:1002600000E000936E0002E000938A0000EA009331
:10027000A30001E00093600001E0009361000DE045
:1002800000939A0000E700EF03BD0FEF00939C007E
:1002900001E000939D0000E00FBB0EBBE29AE09AE4
:1002A0000DB30093AF000FEF0093BB000093BC00B1
:1002B00000E10093BD0000E00093AD0003E0009377
:1002C000AE0000E00093A40003E00093A50000E06E
:1002D0000093A60000E00093AA0000E00093AB00AA
:1002E00000E80FBF02E807BF00E0F02EAC980E94C4
:1002F0000F040E940F040E940F040E940F04AC9A86
:1003000096980E940F040E940F040E940F040E94FE
:100310000F04969AAC9810E10E94E6050E94FA0537
:1003200000E0A02F01E0B02F00E002990BC0000018
:1003300000000000000000000A950000B1F70E94D4
:10034000A4070CC001990AC00000000000000000D2
:1003500000000A950000B1F70E945807AD98AD9AC9
:1003600025E09198E894F7F8869B0CC00E946006FF
:10037000029B0E940606A998AB980499F7CF0091BA
:1003800011000CB901990C94C7016894F0F80E940F
:100390002504029B0E940606049B04C00E9460067E
:1003A0000C94C2010E9462060E946206F7FEEACF28
:1003B0000E941B02F1FE0DC000E00093AD0003E0BF
:1003C0000093AE000E9403020E941B02F1FE01C0D6
:1003D000F9CF00E00093AD0003E00093AE0000E031
:1003E0000093A40003E00093A500E894F1F800E076
:1003F0000093A6000E94A70230E12FEF00911100A8
:100400000CB90C94C201EF93FF930F93E091AD00F0
:10041000F091AE00A190E093AD00F093AE0000919A
:10042000A6000A9511F4E894F1F80093A6000F9144
:10043000FF91EF9108950A2D0B3131F400E0A02FC8
:1004400001E0B02F8AC06CC00A2D0C3019F500E015
:100450000093AB00009113000CB9F5FE13C00E948D
:10046000FA05F5FE07C00E94FA0511E00E94E605B4
:10047000F5FCF5CF00E00093AB00F0FC08950E947E
:1004800048070895F0FC0C9406060E941C06A998E3
:10049000AB9808950A2D0A3019F40E944D0408956E
:1004A0000D3029F400E0A02F01E0B02F08950231B3
:1004B00089F40E9492020A2D063461F50E9492028C
:1004C0000A2D0770013019F46894F3F80895E89440
:1004D000F3F808950D3121F50E9492020A2D02349D
:1004E000E9F40E9492020A2D0770002E0CE0E02F22
:1004F00005E0F02F002DE00F00E0F01FC895002D63
:1005000009B900E0A02F01E0B02F0895BFBFBF5F81
:100510002F170F0702E10D930C9490020DE10D933C
:10052000AD920895F1FE03C00E94030208950E9457
:10053000A70230E2232E3FEF2FEFF7FE01C0089510
:100540002A95D9F73A95C9F72A94B9F70895AD983D
:100550009198E894F7F8AD9A08950E9492020A2DB6
:100560000734C9F508E2A02F01E0B02F0E949202E3
:100570000A2D0F70002E0AE00E94CF0660936400DF
:100580000E9492020A2D0F70002E00916400000D4F
:100590000093640006E3001A20F000E30C94D302F9
:1005A0000895009164000E949202AD920A950000A5
:1005B000D1F701E0702E01E0602E6894F2F80FECA4
:1005C00006B9009113000CB90091AB0000FD3ED3B9
:1005D0000E9471040895083559F40E9492020A2D70
:1005E000077000938A0000E0A02F01E0B02F08956B
:1005F000013489F40E9492020A2D07700093600072
:100600000E9492020A2D07700093610000E0A02F63
:1006100001E0B02F08950D34C9F40E9492020A2D12
:100620000F70002E0AE00E94CF0660936B000E94BC
:1006300092020A2D0F70002E00916B00000E0092A6
:100640006B0000E0A02F01E0B02F08950B37D1F52B
:100650000EE0009364006894F6F80E9492020A2D5E
:100660000D3739F500916400013011F4E894F6F883
:1006700000E0A02F01E0B02F0BE8C02F00E0D02F4A
:100680002DE00D910F7009932A950000D1F7F6FC2B
:100690000C9453030E94530B009397000091130096
:1006A0000CB90C94210C0E948A0B009392000C94BC
:1006B000210CAD92009064000A9400926400000046
:1006C00061F60895043469F40E9492020A2D0F70B5
:1006D00000936C0000E0A02F01E0B02F0E94C00545
:1006E00008950035D9F40E9492020A2D0F70002E51
:1006F0000AE00E94CF0660936D000E9492020A2DCC
:100700000F70002E00916D00000E00926D00689435
:10071000F4F800E0A02F01E0B02F0895013589F42E
:100720000E9492020A2D0F700E9492020A2D0F70F1
:100730000E9492020A2D0F7000E0A02F01E0B02F5E
:100740000895063449F40E9492020A2D0F7000E0C9
:10075000A02F01E0B02F0895033549F40E949202C2
:100760000A2D0F7000E0A02F01E0B02F0895023590
:1007700049F40E9492020A2D0F7000E0A02F01E0C0
:10078000B02F08950E3441F50E9492020A2D0F7089
:10079000002E0AE00E94CF066093A2000E949202FF
:1007A0000A2D0F70002E0091A200000E0092A200F0
:1007B000202D222361F0009113000CB910E20E9459
:1007C000E6050E94FA052A95C9F70E94FA0500E09D
:1007D000A02F01E0B02F08950635E1F40E949202A7
:1007E0000A2D0F70002E0AE00E94CF066093A3002E
:1007F0000E9492020A2D0F70002E0091A300000E9D
:1008000008E00E94CF066093A30000E0A02F01E063
:10081000B02F089500E0A02F01E0B02F08952FEF32
:100820003FEF2A950000E9F73A950000D1F72FEF46
:100830003FEF2A950000E9F73A950000D1F70895B7
:1008400020E52A950000E9F708950091BB000A957C
:10085000D9F40FEF0093BB000091BC000A95B9F4E6
:100860000FEF0093BB000093BC000091BD000A9500
:1008700089F4A998AB980FEF0093BB000093BC00DC
:1008800000E10093BD0008950093BB00089500931C
:10089000BC0008950093BD000895009113000CB9A9
:1008A0000091AB0000FDD2D10FEC06B900E000933F
:1008B00068000AE1602E0F2D047021F001E0602E27
:1008C0000C94710497D118E081D1709061000E945E
:1008D00092090C946B0400916800039503950093B2
:1008E0006800F2FE02C00E9492090FEC06B982D1A4
:1008F00014E06CD10E9464067A94000091F76A9427
:1009000021F70F2D047001F400E0A02F01E0B02FBB
:1009100037D100E7E894F2F8F7F86CD107E006B9B0
:1009200000B30072E9F7089500916D00003021F0E6
:100930000A9500936D000895E894F4F8089508E28C
:10094000C02F01E0D02F00E3102E099105750FB9DB
:100950000EB10078E9F31A940000B9F700B3007201
:10096000E9F79398000000000000939A089508E2C8
:10097000C02F01E0D02F00E3102E09910A7A0FB9A1
:100980000EB10078E9F31A940000B9F700B30072D1
:10099000E9F79398000000000000939A089508E298
:1009A000C02F01E0D02F00E3102E099103700FB982
:1009B000779BFECF1A940000C1F78599FECF9398DC
:1009C000000000000000939A08950FE6C02F01E098
:1009D000D02F00E3902E0881002E00E0099302E45E
:1009E000E02F0AE0F02FE00D00E0F01F002DC89589
:1009F0008894500CA8F00FB9779BFECF9A94000012
:100A000051F78599FECF9398000000000000939A5B
:100A1000052D0C3911F00E9464060FEF089500E0D7
:100A20000FB9779BFECF9A940000C9F78599FECF46
:100A30009398000000000000939A0E94640600E072
:100A400008950001010201020203010202030203F0
:100A50000304010202030203030402030304030468
:100A60000405010202030203030402030304030456
:100A70000405020303040304040503040405040538
:100A80000506010202030203030402030304030434
:100A90000405020303040304040503040405040518
:100AA0000506020303040304040503040405040506
:100AB00005060304040504050506040505060506E8
:100AC00006070102020302030304020303040304F2
:100AD00004050203030403040405030404050405D8
:100AE00005060203030403040405030404050405C6
:100AF00005060304040504050506040505060506A8
:100B000006070203030403040405030404050405A3
:100B10000506030404050405050604050506050687
:100B20000607030404050405050604050506050675
:100B30000607040505060506060705060607060757
:100B4000070808E2C02F01E0D02F0FE6A02F01E038
:100B5000B02F00E309900D920A950000D9F708958F
:100B600000E0002E0EE20FB80000779BFDCF0A9543
:100B70000000C9F79398000000000000939A0895C0
:100B800000E0E02F01E0F02F00E0002E01920F2F97
:100B90000130E1F70E2F0E36C9F708950D920B2F95
:100BA0000130E1F70A2F0E36C9F7089501920F2F91
:100BB0000230E1F70E2F0330C9F708950CE0002E44
:100BC0000CB800005E9908950C94E1050CEFE02F3D
:100BD0000BE0F02F00916300E00F00E0F01FC895DC
:100BE000002D0F70002E05B3007F000E05BA0BE03C
:100BF00005BD089505B50770E9F708950E0E0F0FAE
:100C00000B0B0A0A69696A6A66666565F0FE0C94F0
:100C10001C0600E00093AB000E94080728EB0E942E
:100C2000FA0514E00E94E6050E94FA052A95B9F734
:100C300008950E94330209C000E00093AB00F5FC68
:100C4000F8CF0E9408070E94320708950E940F04FF
:100C50000E940F040E940F04009163000A95009304
:100C6000630024E90E94FA0514E00E94E6050E9450
:100C7000FA052A95B9F700E00093AB000E940F0433
:100C80000E940F040E940F040E940F040E940F0490
:100C90000E94FA05009163000395009363000E948F
:100CA000FA0510E20E94E6050E94FA0500EF03BD76
:100CB000089503B5005B18F003B5045003BD089513
:100CC00096980895969A089500B30072E9F702E2A3
:100CD000E02F0DE0F02F00919C0000909D00069405
:100CE00007950694079506950695E00F00E0F01F1E
:100CF000C895002D0694069420916C00F2FE01C068
:100D0000220F000D20F02A950000D9F701C00FEF47
:100D100001BF0EE003BF0E9420040E942004959AA8
:100D200008950708090A0B0C0D0E16181A1C1E212F
:100D300023242527282A2B2D2F30313233343739DD
:100D40003A3B3C3D3E4041424344464748494A4B7A
:100D50004C4D4F5052545557595B5C5E606264670E
:100D6000696DF3FE06C006E4E02F05E5F02F0C9454
:100D7000BD060AE7E02F01E2F02F04E30E94CF0650
:100D800000916800E00F00E0F01FE60FF51FC89526
:100D9000009287003196C89500928800089528E057
:100DA00050E060E070E0069520F0000C771F0C9496
:100DB000DE060000600D571F000C771F2A9500000B
:100DC00091F708950020E1F00023D1F060E070E099
:100DD000502D500B40F06395000F10F00C94E80676
:100DE00007950C94F606662359F00695000A18F448
:100DF00088940C94FC060894771F6A95000099F774
:100E000008950AE0302E00E3002E0E944508089560
:100E100000E00093AB00F5FC26CB35E020E8059B15
:100E20000DC00E94FA0512E00E94E6050E94FA0534
:100E30002A95A9F73A9599F714C008952CE30599D6
:100E40000BC00E94FA0512E00E94E6050E94FA0516
:100E50002A95A9F706C0089514E00E94E6050E94AD
:100E6000FA050895F0FC089500E00093AB0033E02C
:100E700020E60E94FA0512E00E94E6050E94FA05AB
:100E80002A95B9F73A95A9F701E00093AB000895C8
:100E9000F0FC089520E00E94FA0512E00E94E605A9
:100EA0000E94FA052A95B9F701E00093AB00089576
:100EB0005FEF6FEF7FEF0E94960753E262E372E20B
:100EC0000E94960755E464E574E40E94960759E889
:100ED00068E978E80E94960751E161E171E10E94BA
:100EE000960753E262E372E20E94960755E464E5D6
:100EF00074E40E94960759E868E978E80E9496072A
:100F000051E161E171E10E94960753E262E372E20E
:100F10000E94960755E464E574E40E94960759E838
:100F200068E978E80E949607C3CF089508E2A02FE9
:100F300001E0B02F08E1A02E5D936D937D93AA94FC
:100F4000D9F70E94D902089500E0002E0E944308BC
:100F500008E1002E0E94430800E3002E0E9443088F
:100F600008E4002E0E94430800E6002E0E94430879
:100F700008E7002E0E94430800E9002E0E94430863
:100F800008EA002E0E9443080E94FA051FEF0E9403
:100F9000E60500EC002E0E94430808ED002E0E949A
:100FA00043080E94C0050FE0302E00EF002E0E9483
:100FB00045080E94FA0510E50E94E6050E94C0055A
:100FC00001E00093600001E0009361000E94FA05D7
:100FD0001DE70E94E6050E94C0050E9463080E946A
:100FE000C0050E9474080E94C0050E94FA051DE712
:100FF0000E94E6050E94FA050E941C06089502E27E
:10100000E02F0DE0F02F00E0A02F01E0B02F0091C5
:101010009D0000630D9300919C0002950F7000638A
:101020000D9300919C000F7000630D9300919C0044
:1010300000909D00069407950694079506950695E1
:10104000E00F00E0F01FC895002D02950F700063BF
:101050000D93002D0F7000630D93002D06940694E0
:10106000069420916C00000D2A950000E1F7002EF7
:1010700002950F7000630D93002D0F7000630D93A8
:101080000E944D04089508E1302E00E0A02F01E0F9
:10109000B02F0E94D3080E944D04089500E0A02FB5
:1010A00001E0B02F00E30D9301E30D9302E30D93F4
:1010B00003E30D9304E30D9305E30D9306E30D9312
:1010C00007E30D93089500E0A02F01E0B02F0AE0A0
:1010D000E02F01E1F02F08E1C8950D9231960A95B5
:1010E000D9F70E944D04089500E0A02F01E0B02F31
:1010F00002E2E02F01E1F02F00E1C8950D92319658
:101100000A95D9F70E944D0408958F8E9092202061
:101110007B8F8E918B85848E828092858B9C8D9B1C
:10112000897D82859091889F2020504C4D2D3131B2
:101130005343918A8E908A91929C202020313036A0
:10114000303001E000938B0005E000938C0000E05C
:1011500000938D0001E000938E0007E000938F0064
:1011600003E00093900008E00093910002E00093F8
:10117000920002E00093930001E00093940001E0EC
:101180000093950001E0009396000E94530B00939A
:1011900097000E94210C0E94FA0510E50E94E605C6
:1011A0000E94C00508950D9203943A940000D9F767
:1011B0000895003009F40895002E00E009930A9480
:1011C0000000E1F708951694C19A10F0C29801C08A
:1011D000C29AC1981694C19A10F0C29801C0C29ADE
:1011E000C1981694C19A10F0C29801C0C29AC198D1
:1011F0001694C19A10F0C29801C0C29AC198169470
:10120000C19A10F0C29801C0C29AC1981694C19AAE
:1012100010F0C29801C0C29AC1981694C19A10F0F9
:10122000C29801C0C29AC1981694C19A10F0C2988F
:1012300001C0C29AC19808950694C19A10F0C2984C
:1012400001C0C29AC1980694C19A10F0C29801C018
:10125000C29AC1980694C19A10F0C29801C0C29A6D
:10126000C1980694C19A10F0C29801C0C29AC19860
:101270000694C19A10F0C29801C0C29AC19806940F
:10128000C19A10F0C29801C0C29AC19808950694FC
:10129000C19A10F0C29801C0C29AC1980694C19A2E
:1012A00010F0C29801C0C29AC1980694C19A10F079
:1012B000C29801C0C29AC1980694C19A10F0C2980F
:1012C00001C0C29AC19808950694C19A10F0C298BC
:1012D00001C0C29AC1980694C19A10F0C29801C088
:1012E000C29AC1980694C19A10F0C29801C0C29ADD
:1012F000C19808950694C19A10F0C29801C0C29A8C
:10130000C1980694C19A10F0C29801C0C29AC198BF
:10131000089505E1202E00E0102E0E94E3082A9493
:10132000D1F70895F2FE0DC008E2A02F01E0B02F22
:1013300040E31D900E94E3084A95D9F70E94AE044D
:10134000089501E0502E00E8402E00916B000E94AD
:10135000D90800916B000E94DD0900E0A02F01E098
:10136000B02F0D900E94B106F3FE12C000916000F4
:101370000130B1F50BE00E94DD09E0F0109087002C
:101380000E94E308009088000E9464090C94B1094F
:10139000009160000130D1F500E10E94DD0950F0BC
:1013A000109087000E94E308109088000E94E308D4
:1013B0000C94B1090E94AE040895242C401A00E058
:1013C000500A08F00895022D003011F40894089591
:1013D000422CC19AC298C1984A94D9F708940895AA
:1013E000023071F506E10E94DD0920F30E94B10A86
:1013F000109070000E94E308109071000E94E308B2
:10140000009072000E941C090C94B1090230C9F5C9
:1014100000E20E94DD0970F20E94B10A1090700093
:101420000E94E308109071000E94E308109072007F
:101430000E94E308109073000E94E3080C94B10925
:101440000330E9F401E20E94DD09E8F10E94C20ADA
:10145000109070000E94E308109071000E94E30851
:10146000109072000E94E308109073000E94E3083D
:1014700010907400C19AC298C1980C94B1090C9450
:10148000670A033011F500E30E94DD09E0F00E94D5
:10149000C20A109070000E94E308109071000E9430
:1014A000E308109072000E94E308109073000E94FD
:1014B000E308109074000E94E308109075000E94E9
:1014C000E3080C94B1090C94DA090C94890A0CE233
:1014D0000E94DD09C0F30E94D70A109070000E949C
:1014E000E308109071000E94E308109072000E94BF
:1014F000E308109073000E94E308109074000E94AB
:10150000E3080090750000E0002E0E9447090C944B
:10151000B10900E40E94DD09B0F20E94D70A1090E0
:1015200070000E94E308109071000E94E308109080
:1015300072000E94E308109073000E94E30810906C
:1015400074000E94E308109075000E94E308109058
:1015500076000E94E308109077000E94E3080C9444
:10156000B109009087000E94F00AB0927000C0920A
:101570007100009088000E94F00AB0927200C09240
:1015800073000895009087000E94090BB0927000CC
:10159000C0927100D0927200009088000E94090BE6
:1015A000B0927300C0927400D092750008950090BC
:1015B00087000E942A0BB0927000C0927100D092F6
:1015C0007200E0927300009088000E942A0BB09293
:1015D0007400C0927500D0927600E0927700089572
:1015E00007FAC7F8C6F806FAC5F8C4F805FAC3F84A
:1015F000C2F804FAC1F8C0F803FAB7F8B6F802FA6C
:10160000B5F8B4F801FAB3F8B2F800FAB1F8B0F8E6
:10161000089507FAD7F8D6F8D5F806FAD4F8D3F82B
:10162000D2F805FAD1F8D0F8C7F804FAC6F8C5F828
:10163000C4F803FAC3F8C2F8C1F802FAC0F8B7F860
:10164000B6F801FAB5F8B4F8B3F800FAB2F8B1F8A0
:10165000B0F8089507FAE7F8E6F8E5F8E4F806FACE
:10166000E3F8E2F8E1F8E0F805FAD7F8D6F8D5F8AB
:10167000D4F804FAD3F8D2F8D1F8D0F803FAC7F8BE
:10168000C6F8C5F8C4F802FAC3F8C2F8C1F8C0F841
:1016900001FAB7F8B6F8B5F8B4F800FAB3F8B2F84A
:1016A000B1F8B0F8089500E0002E50918C00050EBE
:1016B00050918E00050E50919000050E50919200B1
:1016C000050E50919400050E50919600050E502D78
:1016D000000C050E602D00E0002E50918B00050ED1
:1016E00050918D00050E50918F00050E5091910084
:1016F000050E50919300050E50919500050E060EB3
:101700000AE0001A10F00C94810B000E0AE0001998
:10171000002E089500E0002E50918B00050E509190
:101720008D00050E50918F00050E50919100050E11
:10173000502D000C050E602D00E0002E50918C0005
:10174000050E50918E00050E50919000050E060E6C
:101750000AE0001A10F00C94A90B000E0AE0001920
:10176000002E089508E2A02F01E0B02F0E94FD0B8B
:101770000E940F0C0E94060C0E941C0C0E94FD0B84
:1017800001EA002E0E94D80B0E94EB0B0D920E94E2
:10179000060C089508E0302E0E94FD0B0E940F0CED
:1017A0000D900E94D80B3A94D9F70E94060C089528
:1017B00008E0000C979808F4979A949A0E941C0CE1
:1017C00094980E941C0C0A95A1F7979A949A0E94EB
:1017D0001C0C9498089508E0949A0E941C0C88941C
:1017E00097990894079494980A95B1F79798949AC2
:1017F0000E941C0C9498979A0895979A949A0E9424
:101800001C0C97980E941C0C949808959798949893
:101810000E941C0C949A0E941C0C979A089500EA4E
:10182000002E0E94D80B00E0002E0E94D80B00E092
:10183000002E0E94D80B089525E02A950000E9F7B4
:10184000089500E000938900F6FC0C942B0C0E9494
:10185000BF0D0C94810C0E94D10E01E0602E00910E
:10186000A300702E6894F2F80091AB0000FDEED951
:101870000E9471040E94B80E01E0602E03E0702EF9
:101880006894F2F80091AB0000FDE0D90E94710469
:1018900000E00093890003E0802E33E00E94400FB7
:1018A00001E0602E01E0702E6894F2F80091AB0028
:1018B00000FDCCD90E9471043A9581F7009189000E
:1018C0000395009389008A9441F704E0802E33E069
:1018D0000E948B0F01E0602E01E0702E6894F2F8F8
:1018E0000091AB0000FDB2D90E9471043A9581F7D6
:1018F000009189000395009389008A9441F70C9424
:10190000D30C01E0602E0091A300702E6894F2F8D1
:101910000091AB0000FD9AD90E9471040E94D70C7F
:1019200001E0602E03E0702E6894F2F80091AB00A5
:1019300000FD8CD90E94710400E00093890003E04F
:10194000802E33E00E94F70C01E0602E01E0702E43
:101950006894F2F80091AB0000FD78D90E94710400
:101960003A9581F7009189000395009389008A9444
:1019700041F704E0802E33E00E945B0D01E0602E11
:1019800001E0702E6894F2F80091AB0000FD5ED982
:101990000E9471043A9581F70091890003950093A4
:1019A00089008A9441F700E000937A00089505E0E9
:1019B00000937B0000E000937C0000937D00009387
:1019C0007E0000937F0000E40093800001E000931C
:1019D000810000E000938200009383000093840064
:1019E0000093850000E5009386000C94780E0BE8C8
:1019F000A02F00E0B02F0E941510000C00927A007A
:101A00000E941510000C102C0E941510000C202CA8
:101A10000E941510000C302C0E941510000C402C58
:101A20000E941510000C502C0E941510000C602C08
:101A300000EA002E0AE0702E05E00E94240E0092BB
:101A40007B0010927C0020927D0030927E004092BC
:101A50007F00509280006092810002E9A02F00E098
:101A6000B02F0E941510102C0E941510202C0E94DF
:101A70001510302C0E941510402C0E941510502C6F
:101A80000E941510602C00E0002E05E0702E06E08C
:101A90000E94520E60908100060C0092810010920C
:101AA0008200209283003092840040928500509200
:101AB00086000C94780E0BE8A02F00E0B02F0E9457
:101AC0001510000C00927A000E941510000C102CCA
:101AD0000E941510000C202C0E941510000C302CB8
:101AE0000E941510000C402C0E941510000C502C68
:101AF0000E941510000C602C00E0002E00E0702EFB
:101B000005E00E94240E00927B0010927C0020923F
:101B10007D0030927E0040927F0050928000609263
:101B2000810002E9A02F00E0B02F0E941510102CB8
:101B30000E941510202C0E941510302C0E941510A8
:101B4000402C0E941510502C0E941510602C00E0B3
:101B5000002E00E0702E06E00E94520E6090810080
:101B6000060C009281001092820020928300309235
:101B7000840040928500509286000C94780E0CE808
:101B8000A02F00E0B02F0E94EE0F000C102C0E943E
:101B9000EE0F000C202C0E94EE0F000C302C0E9447
:101BA000EE0F000C402C0E94EE0F000C502C0E94F7
:101BB000EE0F000C602C00EA002E0AE0702E05E00B
:101BC0000E94240E00927B0010927C0020927D00E7
:101BD00030927E0040927F0050928000609281009F
:101BE00002E9A02F00E0B02F0E942910000C102C59
:101BF0000E942910000C202C0E942910000C302C6F
:101C00000E942910000C402C0E942910000C502C1E
:101C10000E942910000C602C00E0002E05E0702EC0
:101C200006E00E94520E60908100060C0092810036
:101C300010928200209283003092840040928500AE
:101C4000509286000C94780E7694679476946794FC
:101C500057947694679457944794769467945794DE
:101C6000479437947694679457944794379427947D
:101C70007694679457944794379427941794000068
:101C8000000000000000000000000000000076944A
:101C900067945794479437942794179407940A9518
:101CA000B1F70895769467947694679457947694F0
:101CB00067945794479476946794579447943794CD
:101CC00076946794579447943794279476946794BE
:101CD000579447943794279417947694679457941D
:101CE000479437942794179407940A95B1F7089569
:101CF00008E2C02F01E0D02F0AE7A02F00E0B02FAC
:101D00000DE0102E00918A00023079F400916B00F2
:101D10000E94D9080D900E94F00AB992C9921A94B3
:101D2000C9F700E10E94D9080895033081F40091B9
:101D30006B000E94D9080D900E94090BB992C992BC
:101D4000D9921A94C1F70AE00E94D9080895009127
:101D50006B000E94D9080D900E942A0BB992C9927B
:101D6000D992E9921A94B9F704E00E94D90808952B
:101D700005E000937B0000E000937C0000937D0071
:101D800000937E0005E000937F0000E00093800058
:101D9000009381000093820005E0009383000C947F
:101DA0001E0F0BE8A02F00E0B02F0E943510000C92
:101DB000102C0E943510000C202C0E943510000CB5
:101DC000302C0E943510000C402C00EA002E0AE056
:101DD000502E05E00E94D60F00927B0010927C00EE
:101DE00020927D0030927E0040927F000FE8A02F6D
:101DF00000E0B02F0E942910000C102C0E94291026
:101E0000000C202C0E942910000C302C0E9429105C
:101E1000000C402C00E0002E05E0502E04E00E9453
:101E2000D60F50907F00050C00927F00109280002A
:101E300020928100309282004092830008E2C02FFD
:101E400001E0D02F0BE7A02F00E0B02F09E0102E0B
:101E500000918A00023031F400916B000E94D90891
:101E60000C948A0E033031F400916B000E94D90863
:101E70000C949B0E00916B000E94D9080C94AB0E41
:101E80000BE8A02F00E0B02F0E941510000C102CC2
:101E90000E941510000C202C0E941510000C302CF4
:101EA0000E941510000C402C00EA002E0AE0502E73
:101EB00005E00E94D60F00927B0010927C002092D9
:101EC0007D0030927E0040927F000FE8A02F00E05E
:101ED000B02F0E941510102C0E941510202C0E946B
:101EE0001510302C0E941510402C00E0002E05E04B
:101EF000502E04E00E94D60F50907F00050C0092F7
:101F00007F001092800020928100309282004092E7
:101F100083000C941E0F0BE8A02F00E0B02F0E944E
:101F20001510000C102C0E941510000C202C0E9483
:101F30001510000C302C0E941510000C402C00E0F5
:101F4000002E00E0502E05E00E94D60F00927B008C
:101F500010927C0020927D0030927E0040927F00A3
:101F60000FE8A02F00E0B02F0E941510102C0E9447
:101F70001510202C0E941510302C0E941510402C9A
:101F800000E0002E00E0502E04E00E94D60F50909A
:101F90007F00050C00927F0010928000209281004B
:101FA00030928200409283000C941E0F5694479406
:101FB000569447943794569447943794279456945C
:101FC0004794379427941794000056944794379475
:101FD0002794179407940A95C1F7089500918B00F0
:101FE0000F70002E02E8E02F00E2F02F0CE00E94BC
:101FF000CF06E60FF51F00918900E00F00E0F01F0B
:10200000009189000395039500938900C895002DE0
:102010003196C895000F001CE02FF02D0D910F7028
:10202000E00F00E0F01FC895089502E2E02F01E202
:10203000F02F0D910F70002E08E00E94CF06E60FE2
:10204000F51F00918900E00F00E0F01FC895000C1B
:1020500008950D910F70002E0AEFE02F00E2F02F8F
:10206000E00D00E0F01FC89508950D910F70002E4F
:102070000EE0E02F01E2F02FE00D00E0F01FC89528
:102080000895871087108710871087108710871092
:1020900087108C1087108C108C10871087108C1074
:1020A0008C1087108C10871087108C108C108C105F
:1020B000871087108C10871087108C108C10871059
:1020C0008C108C10871087108C1087108C108C103F
:1020D0008C108710871087108C1087108C10871039
:1020E0008C1087108C1087108C108C108710871024
:1020F0008C108C1087108C10871027331B211D39F2
:102100000511091727331B211D3905110917584CD3
:10211000645E62467A6E766872666C425C4E5044CB
:1021200048740E11191513110E0002030202020267
:1021300007000E11100C02011F001F10080C1011D7
:102140000E00080C0A091F0808001F010F101011CB
:102150000E001C02010F11110E001F1008040202D4
:1021600002000E11110E11110E000E11111E100899
:1021700007000E11191513110E00000000000000D9
:10218000000000000000000000000000000000004F
:10219000000000000000000000000000000000003F
:1021A000000000000000000000000000000000002F
:1021B000000000000000C003F00F781E1C386C36D1
:1021C000666606600660366C1668366C6E76CC33D2
:1021D0001C38781EF00FC003000000000000000053
:1021E00000000000000000000000C003F00FF81F16
:1021F0009C399C399E79FE7FFE7FC243E667CE7391
:102200008E713C3CFC3FF81FF00FC0030000000043
:10221000000000000000000000000000381C7C3EB0
:102220007E7EFE7FFE7FFE7FFC3FFC3FF81FF81F97
:10223000F00FF00FE007E007C003C003800180014A
:10224000000000000000000000000000000000008E
:1022500080018001C003E007E007F00FF81FFC3F9A
:10226000FE7FFE7FFC3FF81FF00FE007E007C00392
:10227000800180010000000000000000000000005C
:10228000000000008001C003E007E007E007E0076E
:10229000C0039819BC3DBE7DFE7FFE7FBE7DBC3D68
:1022A00088118001C003C00300000000000000008E
:1022B000000000000000000080018001C003C00396
:1022C000E007E007F00FF00FF81FFC3FFC3FFE7F38
:1022D000BE7D9E798C318001C003C00300000000E8
:1022E00000000000000000000000000000000000EE
:1022F000000000008001E007F00FF81FF81FFC3F0E
:10230000FC3FFC3FFC3FFC3FFC3FF81FF81FF00F79
:10231000E0078001000000000000FFFFFFFFFFFF5B
:10232000FFFFFFFFFFFFFFFFFFFF1FF80FF00FF0A2
:1023300007E007E007E007E007E007E007E00FF04D
:102340000FF01FF8FFFFFFFFFFFFFFFFFFFF000081
:1023500000000000000000000000C003F00F781E25
:102360001C380C300E700660066006600660066061
:1023700006600E700C301C38781EF00FC003000091
:102380000000FFFFFFFFFFFFFFFFFFFFFFFFFFFF5B
:10239000FFFF1FF887F1E3C7F3CFF3CFF3CFF3CFFE
:1023A000F3CFF3CFF3CFF3CFE3C787F11FFCFFFFEA
:1023B000FFFFFFFFFFFF0000000000000008000F0C
:1023C000C01FC03C00360066000600070003F00393
:1023D000FC071C070E0E060C060C060C0E0E1C0746
:1023E000FC07F001000000000000000000000000F9
:1023F000E003F80F380E1C1C0C180C180C181C1CD1
:10240000380EF80FE003C001C001C001E003F80F6F
:10241000F80FC001C001C001000000000000000072
:10242000C000C000C001C001C003C007C00EC00C86
:10243000C01CC018C018C018C018C018C018F000C0
:10244000F800FC00FC00FC007C00380000000000EC
:102450000000E000E001E0036007600EE01CE0190E
:10246000E01B601F601E601C6018601878187C18E4
:102470007E187E187E183E181C1E001F801F801FAD
:10248000801F000F00000000000000000000C001DD
:10249000CC19CC19F80FF007780E3F7C1F78380C58
:1024A000780EF007F80FCC19CC19C001000000001D
:1024B000000000000000000000000000000000001C
:1024C0000000000002000E003E007E00FE01FE073C
:1024D000FE1FFE3FFE1FFE07FE017E003E000E00B7
:1024E00002000000000000000000000000000000EA
:1024F000000000000000000000200038003E003F07
:10250000C03FF03FFC3FFE3FFC3FF03FC03F003F7D
:10251000003E003800200000000000000000000025
:1025200000000000C000E001F003D806CC0CC40895
:10253000C000C000C000C000C000C000C000C0009B
:10254000C000C000C000C000C408CC0CD806F00316
:10255000E001C0000000783C783C783C783C783C56
:10256000381C381C381C381C381C381C381C381CCB
:10257000381C000000000000381C7C3E7C3E381CEB
:1025800000000000000000000000E07FF87FFC1F5A
:102590007C1C7E1C7E1C7E1C7E1C7E1C7C1C7C1C71
:1025A000781C701C701C701C701C701C701C701CC3
:1025B000701C701C701C701C0000000000000000EB
:1025C0000000C003E007700C300C30007000E00029
:1025D000E0033007180E181C181838187018E00C93
:1025E000C0070007000E000C300C300EE007C003DF
:1025F00000000000000000000000000000000000DB
:1026000000000000000000000000000000000000CA
:102610000000000000000000FC1FFC1FFC1FFC1F4E
:1026200000000000000080018001C003E007B00D41
:10263000981988118001800180018001800180014A
:1026400080018001800188119819B00DE007C00356
:10265000800180010000FC3FFC3FC000C000E001A1
:10266000F003D806CC0CC408C000C000C000C000F5
:10267000C000C000C000C000C000C000C000C0005A
:10268000C000C000C000C000C000C000C000C0004A
:10269000C000C000C000C000C000C000C000C0003A
:1026A000C000C000C000C000C000C000C000C0002A
:1026B000C000C000C408CC0CD806F003E001C00084
:1026C000C000000000000000000080018003000343
:1026D0000006000CFF1FFF1F000C00060003800314
:1026E0008001000000000000000000000000000069
:1026F00000000000000000000000000000000000DA
:102700003000380018000C000600FF1FFF1F0600F5
:102710000C0018003800300000000000000000002D
:1027200000000000000000000000000000000000A9
:102730000000000000000000000000000000000099
:102740000000000000000000000000000C000C0071
:102750000C000C00FC1FFC1F00000000000000002B
:1027600000000000000000000000180618060C0C15
:1027700004080618FF3FFF3F061804080C0C180653
:10278000180600000000000000000000000000002B
:102790000000000000000000000000000000000039
:1027A000000080008000C001C001E003E003E003FE
:1027B000F007F007F80FF80FFC1FFC1FFE3FFE3F6D
:1027C000000000000000000000000000FE3FFE3F8F
:1027D000FC1FFC1FF80FF80FF007F007E003E00301
:1027E000E003C001C0018000800000000000000084
:1027F00000000000000000000000000000000000D9
:1028000000000000000000000000000000000000C8
:1028100000000000000000000000000000000000B8
:1028200000000000000000000000000000000000A8
:1028300000000000C003C003C003C003C003C00108
:10284000C001C001C001C001C001C001C001C00180
:1028500000000000C001E003E003C0010000000030
:102860000000000000000000380E380E380E380E50
:10287000380E380E380E380E380E000000000000FA
:102880000000000000000000000000000000000048
:10289000000000000000000000000000E01CE01C40
:1028A000600C700E700E3006FC3FFC3F300638079F
:1028B0001803FE1FFE1F18039C039C038C018C0150
:1028C000CE01CE01000000000000C000C000C0002A
:1028D000E003F807F80FFC06DC00DC00F800F80065
:1028E000F003C007C00FC01EC01CC038C038C038BD
:1028F000CC1CDE1EFC0FF807F003C000C000000077
:10290000000000003C003E007F0067006300733859
:102910007F3E3E0F9E07C001F0007C1E1F1F8F3FB1
:10292000833380318039803F001F000F000000009A
:102930000000000000000000F000F801FC039C0310
:102940009C039C039C01F80078007000FC38DC3884
:10295000DE39CE1B8E1B0E1F0E1EFC3FFC3BF030E3
:10296000000000000000000000000000E000E000A7
:10297000E000E000E000E000E000E000E000000037
:102980000000000000000000000000000000000047
:102990000000000000000000000080078003C0016C
:1029A000E001E000F000700070007800780038006E
:1029B00038003800380038003800380078007800D7
:1029C00070007000F000E000E001C0018003F00042
:1029D000E000C001C0038003800700070007000F6C
:1029E000000F000E000E000E000E000E000E000E76
:1029F000000F000F0007000780078003C003C0011D
:102A0000E000000000000000000000000000C00026
:102A1000C000C000C408DE1EF807C000E00130039B
:102A200018061C0E08040000000000000000000052
:102A30000000000000000000000000000000000096
:102A40000000E000E000E000E000FE0FFE0FFE0FDF
:102A5000E000E000E000E0000000000000000000F6
:102A60000000000000000000000000000000000066
:102A70000000000000000000000000000000000056
:102A80000000000000000000000000000000000046
:102A90000000E003E003E001E001F000F0000000CE
:102AA0000000000000000000000000000000000026
:102AB00000000000F80FF80FF80F00000000000001
:102AC0000000000000000000000000000000000006
:102AD00000000000000000000000000000000000F6
:102AE00000000000000000000000000000000000E6
:102AF0000000000000000000C001E003F007F00744
:102B0000E003C0010000000000000000000C000C09
:102B1000000E00060007000380038001C001C00111
:102B2000E000E000600070003000380018001C0079
:102B30000C000C000000000000000000000000007D
:102B4000C001F007F80F380E3C1E1C1C1C1C1C1C7E
:102B50001C1C1C1C1C1C1C1C1C1C1C1C1C1C3C1E93
:102B6000380EF80FF007C001000000000000000060
:102B700000000000C001F001F801F801C001C0012F
:102B8000C001C001C001C001C001C001C001C0013D
:102B9000C001C001C001F80FF80FF80F00000000DD
:102BA0000000000000000000E003F80FF80F3C1EDA
:102BB0001C1C1C1C001C000E000F8007C003E00141
:102BC000F00078003C001C001C00FC1FFC1FFC1FD8
:102BD000000000000000000000000000E003F00F13
:102BE000F80F381E001C001C001C001CC00FC00386
:102BF000C00F001E001E001C001C1C1C3C1EF80FF9
:102C0000F80FE003000000000000000000000000DA
:102C10008007C007C007E007600770077007380724
:102C200038071C071C070E070E07FE1FFE1FFE1F9E
:102C30000007000700070007000000000000000078
:102C400000000000F80FF80FF80F380038003800C7
:102C5000F803F80FF80F381E001C001C001C001CA5
:102C6000001C1C1C3C1EF80FF807E00300000000CD
:102C70000000000000000000E007F01FF81F38000F
:102C800038001C00DC03FC0FFC0F3C1E1C1C1C1C31
:102C90001C1C1C1C1C1C1C1C380EF80FF007E0032D
:102CA000000000000000000000000000FC0FFC0F0E
:102CB000FC0F000E000F0007000780078003800351
:102CC000C001C001E001E000E000F0007000700011
:102CD0003800380000000000000000000000000084
:102CE000E003F80FF80F3C1E1C1C1C1C1C1C3C1E97
:102CF000F80FF007F007F80F3C1E1C1C1C1C1C1CD6
:102D00003C1EF80FF80FE003000000000000000078
:102D100000000000E003F007F80F380E1C1C1C1C1C
:102D20001C1C1C1C1C1C1C1C3C1EF81FF81FE01D3E
:102D3000001C001C0C1EFC0FFC07F0030000000030
:102D40000000000000000000000000000000C001C2
:102D5000E003E003C00100000000000000000000EC
:102D600000000000C001E003E003C001000000001B
:102D70000000000000000000000000000000000053
:102D80000000C001E003E003C001000000000000FB
:102D90000000000000000000C003C003C001C0012B
:102DA000E000E00060007000000000000000000093
:102DB000000000000000001C001FE01FF803FE00E0
:102DC0001F0007001F00FE00F803E01F001F001C8B
:102DD00000000000000000000000000000000000F3
:102DE000000000000000000000000000FC1FFC1FAD
:102DF0000000000000000000FC1FFC1F000000009D
:102E000000000000000000000000000000000000C2
:102E100000000000000000000000000000000700AB
:102E20001F00FF00F803E00F001F001C001FE00F51
:102E3000F803FF001F000700000000000000000072
:102E400000000000000000000000E003F007F80FA1
:102E5000300E000E000E000F8007C003C001E0001E
:102E6000E000E000E000000000000000E001F003EE
:102E7000F003E00100000000000000000000E0019D
:102E8000F807F80F1C0E1C1C0E1C8E1FCE1FCE1F29
:102E9000EE19EE18EE18EE18EE1CCE1F8E0F1C0069
:102EA0001C00FC01F803E00300000000000000002B
:102EB00000000000800380038003C007C007C00734
:102EC000E00EE00EE00EE00E701C701CF01FF01F14
:102ED000F83F383838381C701C701C700000000037
:102EE0000000000000000000FC01FC073C071C0E75
:102EF0001C0E1C0E1C0E3C0FFC07FC03FC073C0EBA
:102F00001C1C1C1C1C1C1C1C3C1EFC0FFC0FFC0372
:102F1000000000000000000000000000E007F00FCB
:102F2000F80F381C3C1C1C1C1C001C001C001C0046
:102F30001C001C001C001C001C1C3C1C381CF80F36
:102F4000F00FE0070000000000000000000000009B
:102F5000FC01FC073C0F1C0E1C1E1C1C1C1C1C1C1A
:102F60001C1C1C1C1C1C1C1C1C1C1C1C1C1C1C1E9F
:102F70003C0FFC0FFC07FC010000000000000000FB
:102F800000000000FC1FFC1FFC1F1C001C001C009C
:102F90001C001C00FC07FC07FC071C001C001C009C
:102FA0001C001C001C00FC1FFC1FFC1F000000007C
:102FB0000000000000000000FC1FFC1FFC1F1C00A4
:102FC0001C001C001C001C00FC07FC07FC071C006C
:102FD0001C001C001C001C001C001C001C001C0011
:102FE000000000000000000000000000E007F00FFB
:102FF000F80F381E3C1C1C001C001C001C001C0090
:103000001C1F1C1F1C1F1C1C1C1C3C1C381EF81FDA
:10301000F037E03300000000000000000000000076
:103020001C1C1C1C1C1C1C1C1C1C1C1C1C1C1C1CE0
:10303000FC1FFC1FFC1F1C1C1C1C1C1C1C1C1C1C27
:103040001C1C1C1C1C1C1C1C0000000000000000A0
:1030500000000000F80FF80FF80FC001C001C00118
:10306000C001C001C001C001C001C001C001C00158
:10307000C001C001C001F80FF80FF80F00000000F8
:103080000000000000000000801F801F801F001C47
:10309000001C001C001C001C001C001C001C001C50
:1030A0001C1C1C1C1C1C1C1C3C1EF80FF80FE003F5
:1030B0000000000000000000000000001C0C1C1EAE
:1030C0001C0F1C079C03DC01FC01FC007C003C0085
:1030D0007C00FC00FC01DC019C039C071C0F1C1EF7
:1030E0001C3C1C3800000000000000000000000034
:1030F0001C001C001C001C001C001C001C001C00F0
:103100001C001C001C001C001C001C001C001C00DF
:103110001C00FC1FFC1FFC1F000000000000000042
:10312000000000000E381E3C1E3C3E3E3E3E3E3E31
:103130007E3F7E3FFE3FEE3BEE3BCE39CE398E38B2
:103140000E380E380E380E380E380E3800000000DB
:1031500000000000000000001C381C383C383C38DF
:103160007C387C38FC38DC38DC39DC399C3B9C3BD7
:103170001C3B1C3F1C3E1C3E1C3C1C3C1C381C3891
:10318000000000000000000000000000E003F00765
:10319000F80F380E3C1E1C1C1C1C1C1C1C1C1C1C70
:1031A0001C1C1C1C1C1C1C1C1C1C3C1E380EF80F60
:1031B000F007E00300000000000000000000000035
:1031C000FC03FC0F3C1E1C1C1C1C1C1C1C1C1C1C83
:1031D0003C1EFC1FFC0FFC031C001C001C001C0000
:1031E0001C001C001C001C0000000000000000006F
:1031F00000000000E003F007F80F380E3C1E1C1C16
:103200001C1C1C1C1C1C1C1C1C1C1C1C1C1C1C1CFE
:103210001C1C3C1E380EF80FF007E007000E000ED5
:10322000001C000000000000FC03FC0FFC0F1C1E33
:103230001C1C1C1C1C1C1C1C1C0FFC0FFC07FC0178
:10324000DC039C039C071C071C0E1C1E1C1C1C3C46
:10325000000000000000000000000000E003F8078C
:10326000F80F3C0E1C003C0078007800F000E003F2
:10327000C007000F000E001E001C001C1C1EFC0FCF
:10328000F80FE00300000000000000000000000054
:10329000FE3FFE3FFE3FC001C001C001C001C001B2
:1032A000C001C001C001C001C001C001C001C00116
:1032B000C001C001C001C00100000000000000000A
:1032C000000000001C1C1C1C1C1C1C1C1C1C1C1CAE
:1032D0001C1C1C1C1C1C1C1C1C1C1C1C1C1C1C1C2E
:1032E0001C1C3C1E780FF80FF007E00300000000E4
:1032F00000000000000000000E380E381E3C1C1CB0
:103300001C1C1C1C380E380E380E380E7007700747
:1033100070077007E003E003E003C001C001C001D3
:103320000000000000000000000000000E380E3811
:103330000E380E380E388E389C1C9C1CDC1DDC1D93
:10334000DC1DDC1DFC1FFC1F380E380E380E380E3D
:10335000380E180C00000000000000000000000003
:103360003C1E380E780F70077007E003C001C001E3
:10337000C001C001C001E003E00370077007380E10
:10338000380E3C1E1C1C1E3C00000000000000000B
:10339000000000001E3C1C1C1C1C380E380E380E91
:1033A000700770076003E003E003C001C001C001C3
:1033B000C001C001C001C001C001C0010000000087
:1033C0000000000000000000FC3FFC3FFC3F001C30
:1033D000000E0007000780078003C001C001E00164
:1033E000E0007000700038003800FC3FFC3FFC3FFC
:1033F000000000000000000000000000F01FF01FAF
:10340000F01F70007000700070007000700070009D
:103410007000700070007000700070007000F01F8D
:10342000F01FF01F0000000000000000000000007E
:1034300038003800380070007000E000E000C00183
:10344000C001C0018003800300070007000E000ECA
:10345000001C001C003800380000000000000000C4
:1034600000000000FC03FC03FC03800380038003D6
:103470008003800380038003800380038003800334
:10348000800380038003FC03FC03FC0300000000B6
:1034900000000000000000008000C001E003F00711
:1034A000380E1C1C0E380630000000000000000022
:1034B000000000000000000000000000000000000C
:1034C00000000000000000000000000000000000FC
:1034D00000000000000000000000000000000000EC
:1034E00000000000000000000000000000000000DC
:1034F00000000000FE7FFE7FFE7F00000000000055
:103500007000F001E007C00F000E00000000000096
:1035100000000000000000000000000000000000AB
:10352000000000000000000000000000000000009B
:103530000000000000000000000000000000F00398
:10354000F807F80F000E000EF00FF80FF80F3C0F01
:103550001C0E1C0E3C0FFC1FF83BF031000000005D
:103560000000000000003800380038003800380043
:103570003800B803F807F80F780E381C381C381CD0
:10358000381C381C381C381C780EF80FDC078C03EC
:10359000000000000000000000000000000000002B
:1035A000000000000000E007F00FF80F380E1C0CC0
:1035B0001C001C001C001C001C001C00381CF81FF8
:1035C000F00FE00700000000000000000000000E07
:1035D000000E000E000E000E000EE00EF00FF80FB1
:1035E000380F1C0E1C0E1C0E1C0E1C0E1C0E1C0E6E
:1035F000380FF81FF01DE018000000000000000068
:103600000000000000000000000000000000E003D7
:10361000F007F80F381E1C1C3C1EFC0FFC071C009A
:103620001C001C003818F81FF01FE0070000000005
:103630000000000000008007C01FE01FE018E0004D
:10364000E000FE0FFE0FE000E000E000E000E00020
:10365000E000E000E000E000E000E000E000E0006A
:10366000000000000000000000000000000000005A
:1036700000000000E018F01DF80F380F1C0E1C0EA3
:103680001C0E1C0E1C0E380FF80FF00FE00E000E73
:10369000000E180FF807F807E001000000001C00FA
:1036A0001C001C001C001C001C00DC03FC0FFC1F89
:1036B0003C1E1C1C1C1C1C1C1C1C1C1C1C1C1C1C28
:1036C0001C1C1C1C1C1C1C1C00000000000000001A
:1036D0000000E000E000E000000000000000FC014D
:1036E000FC01FC01C001C001C001C001C001C0015A
:1036F000C001C001C001C001C001C0010000000044
:103700000000800380038003000000000000E00F41
:10371000E00FE00F000E000E000E000E000E000E77
:10372000000E000E000E000E000E1C0E1C0E1C0ED5
:103730003807F807F003000000000E000E000E002E
:103740000E000E000E000E1E0E0F8E07CE03CE01D1
:10375000EE007E007E00FE00EE00CE018E038E079E
:103760000E0F0E1E00000000000000000000FC0113
:10377000FC01FC01C001C001C001C001C001C001C9
:10378000C001C001C001C001C001C001C001C00131
:10379000C001C001C001C001000000000000000025
:1037A0000000000000000000000000000000E738FA
:1037B000F77DFEFF9EF38EE38EE38EE38EE38EE3D2
:1037C0008EE38EE38EE38EE38EE38EE30000000053
:1037D00000000000000000000000000000000000E9
:1037E00000008C0FDC1FD83F783C38383838383828
:1037F0003838383838383838383838383838383849
:1038000000000000000000000000000000000000B8
:10381000000000000000E003F007F80F380E1C1C49
:103820001C1C1C1C1C1C1C1C1C1C1C1C380EF80FFB
:10383000F007E003000000000000000000000000AE
:10384000000000000000000000008C03DC07F80FFF
:10385000780E381C381C381C381C381C780EF80FB1
:10386000D807980338003800380000000000000036
:103870000000000000000000000000000000E01850
:10388000F01DF80F380F1C0E1C0E1C0E1C0E1C0E0B
:10389000380FF80FF00FE00E000E000E000E0000C3
:1038A0000000000000000000000000000000000018
:1038B00000009E07DC0FFC1F781C781C38003800C5
:1038C0003800380038003800380038003800380038
:1038D00000000000000000000000000000000000E8
:1038E000000000000000F003F807FC071C060C00B5
:1038F0001C00FC00F803E007000F000E0C0EFC0F8C
:10390000FC07F003000000000000000000000000C1
:103910000000E000E000E000E000FC0FFC0FFC0F06
:10392000E000E000E000E000E000E000E000E0187F
:10393000E01CE01FC00F8007000000000000000036
:1039400000000000000000000000000000001C0E4D
:103950001C0E1C0E1C0E1C0E1C0E1C0E1C0E1C0E17
:103960001C0E1C0E3C0FF80DF81DF0180000000096
:103970000000000000000000000000000000000047
:1039800000001C1C3C1E380E380E380E70077007E5
:1039900070077007E003E003E003C001C001C0014D
:1039A0000000000000000000000000000000000017
:1039B000000000000000077007700770CE39CE3994
:1039C000EE3B6E3B6C1B7C1F7C1F3C1E3C1E380E6E
:1039D000180C180C0000000000000000000000009F
:1039E000000000000000000000003C1E380E780FB0
:1039F0007007E003E003C001C001E003E0037007CB
:103A0000780F380E1C1C1E3C000000000000000057
:103A1000000000000000000000001C703C783838F6
:103A20003838781C701C701C700CE00EE00EE0063C
:103A3000C007C007C007800380038003C601FE01E2
:103A4000FC0000000000000000000000000000007A
:103A50000000FC1FFC1FFC0F000780078003C00153
:103A6000E001E000700078003800FC1FFC1FFC1F24
:103A700000000000000000078007C007C001C0016F
:103A8000C001C001C001C001C001C001FC007C0038
:103A90007C00C000C001C001C001C001C001C00164
:103AA000C001C001C007800700070000C001C001BD
:103AB000C001C001C001C001C001C001C001C001FE
:103AC000C001C001C001C001C001C001C001C001EE
:103AD000C001C001C001C001C001C00100007800E8
:103AE000F800F801C001C001C001C001C001C0015F
:103AF000C001C001800F000F800FC001C001C001D4
:103B0000C001C001C001C001C001C001F801F8003E
:103B100078000000000000007830FE38FE3F861F6D
:103B2000000F000000000000000000000000000086
:103B30000000000000000000000000000000000085
:103B40000000000000000000000000000000000075
:103B50000000000000000000000000000000000065
:103B60000000000000000000000000000000000055
:103B70000000000000000000000000000000000045
:103B8000800380038003C007C007C007E00EE00E7B
:103B9000E00EE00E701C701CF01FF01FF83F38386C
:103BA00038381C701C701C70000000000000000001
:103BB00000000000FC1FFC1FFC1F1C181C001C0048
:103BC0001C001C00FC03FC07FC0F3C1E1C1C1C1CE6
:103BD0001C1C1C1C3C1EFC0FFC0FFC030000000006
:103BE0000000000000000000FC01FC07FC073C0F87
:103BF0001C0E1C0E1C0E3C0FFC07FC03FC073C0FAC
:103C00001C1E1C1C1C1C1C1C3C1EFC0FFC0FFC0363
:103C1000000000000000000000000000FC1FFC1F6E
:103C2000FC1F1C181C181C001C001C001C001C0085
:103C30001C001C001C001C001C001C001C001C00A4
:103C40001C001C000000000000000000000000003C
:103C5000000F800F800FC00FC00FE00FE00EE00ECE
:103C6000E00E700E700E700E700E380E380E380E9C
:103C7000380EF80FFE3FFE3F063006300000000011
:103C800000000000FC1FFC1FFC1F1C001C001C008F
:103C90001C001C00FC07FC07FC071C001C001C008F
:103CA0001C001C001C00FC1FFC1FFC1F000000006F
:103CB0000000000000000000C771C771C771CE3955
:103CC000CE39CE39DC1DDC1DF80FF007F007F80FF8
:103CD000DC1DDC1DCE39CE39CE39C771C771C77135
:103CE000000000000000000000000000C001F0071C
:103CF000F00F380E180E000E000E000EC007E00385
:103D0000E007000E001C001C001C0C1C1C1CFC1FEF
:103D1000F80FF007000000000000000000000000A5
:103D20001C381C381C3C1C3C1C3E1C3E1C3F1C3BD5
:103D30009C3B9C3BDC39DC39DC38FC387C387C38FB
:103D40003C383C381C381C38000000000000C00320
:103D5000C00300001C381C381C3C1C3C1C3E1C3E94
:103D60001C3F1C3B9C3B9C3BDC39DC39DC38FC3881
:103D70007C387C383C383C381C381C38000000004B
:103D800000000000000000001C1C1C1C1C0E1C0776
:103D90009C03DC01FC01FC007C003C007C00FC007E
:103DA000FC01DC019C031C071C0E1C1C1C381C386D
:103DB000000000000000000000000000003FC03FC5
:103DC000C03FE039E038E038E038F038703870381B
:103DD0007038783838383838383838381C381C3823
:103DE0001C381C380000000000000000000000002B
:103DF0000E701E781E783E7C3E7C3E7C7E7E6E760B
:103E0000EE77CE73CE73CE738E710E700E700E7011
:103E10000E700E700E700E700000000000000000AA
:103E2000000000001C381C381C381C381C381C389A
:103E30001C381C38FC3FFC3FFC3F1C381C381C382D
:103E40001C381C381C381C381C381C38000000007A
:103E50000000000000000000E007F00FF81F381C11
:103E60001C381C381C381C381C381C381C381C38B2
:103E70001C381C381C381C38381CF81FF00FE007A1
:103E8000000000000000000000000000FC3FFC3FBC
:103E9000FC3F1C381C381C381C381C381C381C389B
:103EA0001C381C381C381C381C381C381C381C3872
:103EB0001C381C380000000000000000000000005A
:103EC000FC07FC1FFC3F3C3C1C381C381C381C38D1
:103ED0001C383C3CFC1FFC0FFC071C001C001C0099
:103EE0001C001C001C001C00000000000000000062
:103EF00000000000E007F00FF81F783C3C381C3849
:103F00001C001C001C001C001C001C001C001C00D1
:103F10001C383C38783CF81FF00FE0070000000028
:103F20000000000000000000FE3FFE3FFE3FC00119
:103F3000C001C001C001C001C001C001C001C00179
:103F4000C001C001C001C001C001C001C001C00169
:103F50000000000000000000000000001C381C38B9
:103F60001C381C381C381C381C381C383C3CFC3FA6
:103F7000F83FE03F003C003800380C381C3CFC3F68
:103F8000F81FF00700000000000000000000000023
:103F9000F007FC1FFE3FEF7BC771C771C771C77188
:103FA000C771C771EF7BFE3FFC1FF007C001C00166
:103FB000C001C001C001C0010000000000000000FD
:103FC000000000003C1E380E780F70077007E003F9
:103FD000C001C001C001C001C001E003E0037007DF
:103FE0007007380E380E3C1E1C1C1E3C00000000E2
:103FF00000000000000000001C1C1C1C1C1C1C1CE1
:104000001C1C1C1C1C1C1C1C1C1C1C1C1C1C1C1CF0
:104010001C1C1C1C1C1C1C1C1C1CFC1FFC3FFC3FF7
:104020000030003000000000000000001C381C3888
:104030001C381C381C381C381C381C381C383C3CBC
:10404000FC3FF83FE03F00380038003800380038C7
:1040500000380038000000000000000000000000F0
:10406000071C071CE71CE71CE71CE71CE71CE71CF8
:10407000E71CE71CE71CE71CE71CE71CE71CE71C28
:10408000E71CFF1CFF1FFF1F0000000000000000D6
:1040900000000000071C071CE71CE71CE71CE71CCE
:1040A000E71CE71CE71CE71CE71CE71CE71CE71CF8
:1040B000E71CE71CE71CFF1FFF3FFF3F00300030FD
:1040C00000000000000000003F003F003F003B00F8
:1040D0003800380038003800F807F81FF83F783CFF
:1040E0003838383838383838783CF83FF81FF8070F
:1040F00000000000000000000000000007700770D2
:104100000770077007700770077007707F70FF7186
:10411000FF73CF738773877387738773CF73FF734F
:10412000FF717F7000000000000000000000000030
:104130001C001C001C001C001C001C001C001C009F
:10414000FC07FC1FFC3F3C3C1C381C381C381C384E
:104150003C3CFC3FFC0FFC030000000000000000A2
:1041600000000000F007F80FF81F3C1C1C381C383A
:1041700000380038C03FC03FC03F0038003800382A
:104180001C381C383C1CF81FF80FF007000000001A
:104190000000000000000000870FC71FE73FE7385E
:1041A000777077707770777077707F707F707770C7
:1041B00077707770777077706730E738C71F870F31
:1041C000000000000000000000000000E03FF83F99
:1041D000FC3F3C3C1C381C381C381C38383CF83F31
:1041E000F03FC03FE039E038F038703838383C38BC
:1041F0001C381E3800000000000000000000000015
:1042000000000000000000000000F803F807F01FA5
:10421000001C001CE01DF81FF81F3C1E1C1C1C1C71
:104220003C1EFC1FF83BF0310000000000000000C5
:104230000000F00FF80F98073800F000E003800747
:10424000E00F701E381C1C381C381C381C381C38F9
:104250001C381C383C3C781EF00FC00300000000E6
:10426000000000000000F003F8071C079C03FC009E
:104270007C00FC01FC073C071C0E1C1C1C1C1C1CAD
:104280001C1C1C1C1C1C1C1C380EF80FF003E0012D
:10429000000000000000000000000000000000001E
:1042A000000000000000F003F807F80F181E001CC3
:1042B000001E800FE003F00038001C001C18FC1FDB
:1042C000F81FE007000000000000000000000000F0
:1042D000F001E007C00F000E001CE01CF01DF81FED
:1042E000381E1C1C1C1C1C1C1C1C1C1C1C1C1C1CF0
:1042F000380EF80FF003E00100000000000000009D
:104300000000000000000000000000000000E007C6
:10431000F00FF81F381C1C383C3CFC3FFC1FFC0F06
:104320000C000C001C18F81FF01FE00F000000002C
:10433000000000000000000000000000000000007D
:104340000000C631CE39CE39FC1FF80FE003FC1F48
:10435000FE3FCE39CE39CE39CE39CE39CE39CE39EF
:10436000000000000000000000000000000000004D
:10437000000000000000E003F007F80F381C181CD4
:10438000000EC007C00FC01F003800381C3CFC1FC7
:10439000F80FF0070000000000000000000000001F
:1043A000000000000000000000001C1C1C1C1C1C65
:1043B0001C1C1C1C1C1C1C1C1C1C1C1C1C1C1C1E3B
:1043C0003C1FFC1FF83DF03800000000000000001A
:1043D0000000000000000000E001E00100001C1CE3
:1043E0001C1C1C1C1C1C1C1C1C1C1C1C1C1C1C1C0D
:1043F0001C1C1C1E3C1FFC1DF83DF038000000007A
:1044000000000000000000000000000000000000AC
:1044100000001C3C1C1E1C0F9C079C03DC01FC00C4
:10442000FC00DC019C031C071C0E1C1C1C381C38E7
:10443000000000000000000000000000000000007C
:10444000000000000000803FC03FE03FE038E0385F
:10445000E038703870387038303838383838383894
:104460001C381C38000000000000000000000000A4
:10447000000000000000000000000E701E783E7C6E
:104480007E7E7E7ECE73CE73CE738E710E700E7076
:104490000E700E700E700E70000000000000000024
:1044A00000000000000000000000000000001C38B8
:1044B0001C381C381C381C38FC3FFC3FFC3F1C38A7
:1044C0001C381C381C381C381C381C3800000000F4
:1044D00000000000000000000000000000000000DC
:1044E0000000E007F00FF81F381C1C381C381C387F
:1044F0001C381C381C381C38381CF81FF00FE0071B
:1045000000000000000000000000000000000000AB
:10451000000000000000FC1FFC1FFC1F1C1C1C1CDA
:104520001C1C1C1C1C1C1C1C1C1C1C1C1C1C1C1CCB
:104530001C1C1C1C0000000000000F0F0F0F0F0FB1
:104540000F0F0F0F000000000000000000000F0F11
:104550000F0F0F0F0F0F0F0F0000000000000000E3
:1045600000000F0F0F0F0F0F0F0F0F0F00000F0F97
:104570000F0F0F0F0F0F0F0FF070F070F070F07043
:10458000F0700F0F0F0F0F0F0F0F0F0FF070F07075
:10459000F070F070F0700F0F0F0F0F0F0F0F0F0F65
:1045A000F070FF7FFF7FFF7FFF7F0F0F0F0F0F0F59
:1045B0000F0F0F0F0F0FFF7FFF7FFF7FFF7F0F0F8B
:1045C0000F0F0F0F0F0F0F0F0F0FFF7FFF7FFF7FDB
:1045D000FF7F0F0F0F0F800180018001800180019C
:1045E00080018001800180018001800180018001C3
:1045F00080018001800180018001800180018001B3
:1046000080018001800180018001800180018001A2
:104610008001800180018001800180018001800192
:10462000800180018001FF01FF0180018001800184
:104630008001800180018001800180018001800172
:104640008001800180018001800180018001800162
:1046500080018001FF01FF01800180018001FF01D5
:10466000FF018001800180018001800180018001C3
:10467000800130063006300630063006300630063F
:1046800030063006300630063006300630063F066B
:104690003F0630063006300630063006300630065B
:1046A0003006300630060000000000000000000068
:1046B00000000000000000000000000000000000FA
:1046C0000000FF07FF0730063006300630063006D0
:1046D00030063006300630063006000000000000CC
:1046E00000000000000000000000000000000000CA
:1046F000FF01FF01800180018001FF01FF018001B6
:1047000080018001800180018001800180013006EC
:1047100030063006300630063006300630063006E9
:10472000300630063F063F060006000600063F063C
:104730003F063006300630063006300630063006BA
:1047400030063006300630063006300630063006B9
:1047500030063006300630063006300630063006A9
:104760003006300630063006300630063006300699
:104770003006300630060000000000000000000097
:10478000000000000000000000000000FF07FF071D
:104790000006000600063F063F06300630063006DB
:1047A0003006300630063006300630063006300659
:1047B0003006300630063006300630063006300649
:1047C0003F063F06000600060006FF07FF07000041
:1047D00000000000000000000000000000003006A3
:1047E0003006300630063006300630063006300619
:1047F00030063006300630063006FF07FF0700009F
:1048000000000000000000000000000000000000A8
:104810000000800180018001800180018001800111
:104820008001800180018001FF01FF018001800182
:104830008001FF01FF0100000000000000000000F7
:104840000000000000000000000000000000000068
:104850000000000000000000000000000000000058
:10486000FF01FF0180018001800180018001800142
:104870008001800180018001800180018001800130
:104880008001800180018001800180018001800120
:1048900080018001800180FF80FF00000000000097
:1048A0000000000000000000000000000000800187
:1048B00080018001800180018001800180018001F0
:1048C00080018001800180018001FFFFFFFF000067
:1048D00000000000000000000000000000000000D8
:1048E00000000000000000000000000000000000C8
:1048F0000000000000000000000000000000FFFFBA
:10490000FFFF800180018001800180018001800122
:10491000800180018001800180018001800180018F
:10492000800180018001800180018001800180017F
:10493000800180FF80FF8001800180018001800173
:1049400080018001800180018001000000000000E2
:104950000000000000000000000000000000000057
:10496000000000000000FFFFFFFF0000000000004B
:1049700000000000000000000000000000008001B6
:10498000800180018001800180018001800180011F
:1049900080018001800180018001FFFFFFFF800115
:1049A00080018001800180018001800180018001FF
:1049B00080018001800180018001800180018001EF
:1049C000800180018001800180FF80FF80018001E3
:1049D000800180FF80FF80018001800180018001D3
:1049E0008001800180013006300630063006300636
:1049F0003006300630063006300630063006300607
:104A0000300630FE30FE3006300630063006300606
:104A100030063006300630063006300630063006E6
:104A200030063006300630063006300630063006D6
:104A300030FE30FE300030003000F0FFF0FF0000AC
:104A40000000000000000000000000000000000066
:104A50000000000000000000000000000000000056
:104A600000000000F0FFF0FF30003000300030FEAA
:104A700030FE30063006300630063006300630068E
:104A80003006300630063006300630063006300676
:104A900030063006300630063FFE3FFE00000000C4
:104AA0000000FFFFFFFF000000000000000000000A
:104AB00000000000000000000000000000000000F6
:104AC000000000000000000000000000FFFFFFFFEA
:104AD0000000000000003FFE3FFE300630063006BA
:104AE0003006300630063006300630063006300616
:104AF0003006300630063006300630063006300606
:104B000030FE30FE30003000300030FE30FE300627
:104B1000300630063006300630063006300600001B
:104B20000000000000000000000000000000000085
:104B300000000000FFFFFFFF000000000000FFFF7B
:104B4000FFFF000000000000000000000000000067
:104B500000003006300630063006300630063006DB
:104B600030063006300630063FFE3FFE00000000F3
:104B700000003FFE3FFE30063006300630063006AD
:104B800030063006300680018001800180018001FE
:104B9000800180018001800180018001FFFFFFFF13
:104BA000000000000000FFFFFFFF00000000000009
:104BB0000000000000000000000030063006300653
:104BC0003006300630063006300630063006300635
:104BD000300630063006FFFFFFFF00000000000037
:104BE00000000000000000000000000000000000C5
:104BF00000000000000000000000000000000000B5
:104C000000000000FFFFFFFF000000000000FFFFAA
:104C1000FFFF80018001800180018001800180010F
:104C20008001000000000000000000000000000003
:104C30000000000000000000000000000000FFFF76
:104C4000FFFF3006300630063006300630063006EC
:104C500030063006300630063006300630063006A4
:104C60003006300630063006300630063006300694
:104C70003006F0FFF0FF0000000000000000000020
:104C800000000000000000000000800180018001A1
:104C9000800180018001800180018001800180010C
:104CA00080FF80FF80018001800180FF80FF000085
:104CB00000000000000000000000000000000000F4
:104CC00000000000000000000000000000000000E4
:104CD0000000000080FF80FF80018001800180FFD4
:104CE00080FF8001800180018001800180018001BE
:104CF0008001000000000000000000000000000033
:104D00000000000000000000000000000000F0FFB4
:104D1000F0FF30063006300630063006300630062A
:104D200030063006300630063006300630063006D3
:104D300030063006300630063006300630063006C3
:104D40003006FFFFFFFF3006300630063006300623
:104D500030063006300630063006800180018001C2
:104D6000800180018001800180018001800180013B
:104D7000FFFFFFFF800180018001FFFFFFFF800137
:104D8000800180018001800180018001800180011B
:104D9000800180018001800180018001800180010B
:104DA00080018001800180018001FF01FF0100007E
:104DB00000000000000000000000000000000000F3
:104DC00000000000000000000000000000000000E3
:104DD00000000000000000000000000080FF80FFD5
:104DE00080018001800180018001800180018001BB
:104DF000800180018001FFFFFFFFFFFFFFFFFFFF3A
:104E0000FFFFFFFFFFFFFFFFFFFFFFFFFFFFFFFFB2
:104E1000FFFFFFFFFFFFFFFFFFFFFFFFFFFFFFFFA2
:104E2000FFFFFFFFFFFFFFFFFFFF0000000000008C
:104E30000000000000000000000000000000000072
:104E40000000000000000000FFFFFFFFFFFFFFFF6A
:104E5000FFFFFFFFFFFFFFFFFFFFFFFFFFFFFF0061
:104E6000FF00FF00FF00FF00FF00FF00FF00FF004A
:104E7000FF00FF00FF00FF00FF00FF00FF00FF003A
:104E8000FF00FF00FF00FF00FF00FF00FF00FF002A
:104E9000FF0000FF00FF00FF00FF00FF00FF00FF1A
:104EA00000FF00FF00FF00FF00FF00FF00FF00FF0A
:104EB00000FF00FF00FF00FF00FF00FF00FF00FFFA
:104EC00000FF00FF00FF00000000000000000000E5
:104ED00000000000000000000000000000000000D2
:104EE00000000000FFFFFFFFFFFFFFFFFFFFFFFFCE
:104EF000FFFFFFFFFFFFFFFFFFFF000000000000BC
:104F000000000000000000000000DC03FC0FFC1F9C
:104F10003C1E1C1C1C1C1C1C1C1C1C1C1C1C1C1CAF
:104F20003C1EFC1FFC0FDC031C001C001C000000CE
:104F30000000000000000000000000000000E0078A
:104F4000F00FF81F381C1C1C1C001C001C001C004F
:104F50001C001C00381CF81FF00FE00700000000C8
:104F60000000000000000000000000000000000041
:104F70000000FE3FFE3FFE3FCE39C001C001C00130
:104F8000C001C001C001C001C001C001C001C00119
:104F90000000000000000000000000000000000011
:104FA0000000000000001C1C1C1C1C1C1C1C1C1CE9
:104FB0001C1C3C1EFC1FF81FF01F001C0C1CFC1FBF
:104FC000F80FF007000000000000000000000000E3
:104FD0000000000000000000C001F007FC1FFE3FC1
:104FE000C771C771C771C771C771FF7FFE3FF80FE7
:104FF000C001C001C001C0010000000000000000AD
:1050000000000000000000000000000000003C3C28
:10501000381C781E700EE007E007C003C003E007ED
:10502000E007700E781E381C1C381E780000000047
:105030000000000000000000000000000000000070
:105040000000070E070E070E070E070E070E070ECD
:10505000070E070E070E070E0F0FFF0FFE3F783EDD
:1050600000380018000000000000000000000000F0
:105070000000000000001C381C381C381C381C388C
:105080001C381C38FC3FF83FE03F0038003800383F
:1050900000380038000000000000000000000000A0
:1050A00000000000000000000000C771C771C77158
:1050B000C771C771C771C771C771C771C771C77130
:1050C000C771FF7FFF7F8E730000000000000000AB
:1050D0000000000000000000000000000000C77198
:1050E000C771C771C771C771C771C771C771C77100
:1050F000C771C771C771FF7FFF7F8E63006000605B
:10510000000000000000000000000000000000009F
:1051100000003F003F00380038003800B803F80FA7
:10512000F81F783C38383838783CF83FF81FF00FD3
:10513000000000000000000000000000000000006F
:10514000000000000000077007700770077007700C
:105150007770FF71FF738F77077707778F77FF7708
:10516000FF73FE710000000000000000000000005E
:10517000000000000000000000001C001C001C00DB
:105180001C001C00DC01FC07FC0F1C1C1C1C1C1C54
:105190001C1CFC1FFC0FF8070000000000000000B2
:1051A0000000000000000000000000000000E0031C
:1051B000F007F80F380E181C001CC01FE01FC01F9E
:1051C000001C181C380EF80FF007E0030000000068
:1051D00000000000000000000000000000000000CF
:1051E0000000870FC71FE73FE738777077707F7041
:1051F0007F70777077707770E738E73FC71F870F4A
:10520000000000000000000000000000000000009E
:10521000000000000000E03FF03F783E3C3C1C38BE
:105220003C3C7C3EF83FE03F803BC039E038703882
:1052300038381C3800000000000098019801000078
:10524000FF07FF07FF070700070007000700070029
:10525000FF00FF00FF00070007000700070007002E
:105260000700FF07FF07FF07000000000000000025
:105270000000000000000000600660060000E0037F
:10528000F007780F380E1C1C3C1E7C1FFC0FFC0323
:105290001C001C00381CF81FF00FE0070000000085
:1052A00000000000000000000000000000000000FE
:1052B0000000000000000000000000000000000EE0
:1052C00000078003C001E000700038001C000E00E1
:1052D00000000000000000000000000000000000CE
:1052E00000000000000000000000000000000000BE
:1052F0001C0038007000E000C00180030007000EB1
:10530000001C003800000000000000000000000049
:105310000038001C000E00078003C001E000700090
:1053200038001C0000000000000000000000000029
:10533000000000000000000000000000000000006D
:10534000000000001C0038007000E000C001800375
:105350000007000E001C00380000000000000000E4
:10536000000000000000000000000000000000003D
:10537000000000000000000000000000000000002D
:1053800080030007000EFC1FFC1FFC1F000E00071F
:10539000800300000000000000000000000000008A
:1053A00000000000000000000000000000000000FD
:1053B00000000000E00070003800FC1FFC1FFC1F14
:1053C00038007000E0000000000000000000000055
:1053D00000000000000000000000000000000000CD
:1053E000000000000000000000000000C001C0013B
:1053F000C001C001C411CC19DC1DF80FF007E00397
:10540000C0010000000000000000000000000000DB
:10541000000000000000000000000000000000008C
:10542000C001E003F007F80FDC1DCC19C411C00166
:10543000C001C001C0010000000000000000000029
:105440000000000000000000000000000000C0019B
:10545000C00100000000FC1FFC1FFC1F000000003A
:10546000C001C001000000000000000000000000BA
:10547000000000000000000000000000C001C001AA
:10548000C001C001C001FE3FFE3FFE3FC001C001A0
:10549000C001C001C001C00100000000FC3FFC3F92
:1054A00000000000000000000000000000000000FC
:1054B0000777075707770F070F071F071F073F07D4
:1054C000370777076707E707C707C707870787070C
:1054D0000707070707070707000000000000000094
:1054E0000000000000000000000006300630E63337
:1054F000F80FFC1F3C1E1C1C1C1C3C1EFC1FF80F44
:10550000E633063006300000000000000000000016
:10551000000000000000000000000000000000008B
:105520000000000000000000F007F007F007000096
:10553000000000000000000000000000000000006B
:10554000000000000000000000000000000000005B
:10555000000000000000000000000000000000004B
:10556000000000000000000000000000000000003B
:105C000070007000700070007000300030003000D4
:105C10003000300030003000300030000000000064
:105C20007000F800F80070000000000000000000A4
:105C30000000000063006300630063006300630012
:105C4000630063006300000000000000000000002B
:105C50000000000000000000000000000000000044
:105C600000000000000000008C018C018C018C0100
:105C70008C018C01FF01FF018400C6004200FF017E
:105C8000FF0163006300630063006300630063005F
:105C900000000000000000000000000018007C0070
:105CA000FF00DB019B001B001B001B001F001E00F0
:105CB0007800F800D801980198019801980199019D
:105CC000DB01FF007E001800000000000000000063
:105CD0000E001F003B003300330033003B039F03E3
:105CE000C601700038009E01C70363033003300310
:105CF000300370036003C0010000000000000000DA
:105D0000000000007800FC008E01860186018601FB
:105D1000C6006C003C0038006E066606C706C30766
:105D20008307030703068E07FE07780600000000BE
:105D30000000000000000000030003000300030057
:105D40000300030003000300030000000000000044
:105D50000000000000000000000000000000000043
:105D600000000000000060003000180018000C0067
:105D70000C000600060006000600030003000300F6
:105D800003000300030003000600060006000600EF
:105D90000C000C00180018000000030006000C00A6
:105DA0000C00180018003000300030003000600097
:105DB0006000600060006000600060003000300043
:105DC00030003000180018000C000C00000000002B
:105DD0000000000000000000000030003000300033
:105DE0003102B703FE0130007800CC008601870342
:105DF00002010000000000000000000000000000A0
:105E00000000000000000000000000000000000092
:105E10003000300030003000FF03FF03300030005E
:105E20003000300000000000000000000000000012
:105E30000000000000000000000000000000000062
:105E40000000000000000000000000000000000052
:105E500000000000000000000000000000003C0006
:105E60003C001C001C000E000000000000000000B0
:105E70000000000000000000000000000000000022
:105E8000FF01FF0100000000000000000000000012
:105E90000000000000000000000000000000000002
:105EA00000000000000000000000000000000000F2
:105EB00000000000000000000000000000000000E2
:105EC0000000000000000E001F001F000E00000078
:105ED00000000000000000000003000380018001BA
:105EE000C000C000600060003000300018001800E2
:105EF00018000C000C00060006000300030003005D
:105F000000000000000000000000000038007C00DD
:105F1000EE00C701830183018301830183018301B3
:105F2000830183018301830183018301C701EE00A3
:105F30007C003800000000000000000000000000AD
:105F400038003F00370030003000300030003000B3
:105F500030003000300030003000300030003000C1
:105F600030003000FF01FF010000000000000000D1
:105F7000000000007C00FE00C60183018301800157
:105F8000800180018001C001E000700038001C0029
:105F90000E00060003000300FF01FF0100000000E7
:105FA00000000000000000007C00FE00C70182012C
:105FB0008001800180018001C0007800F800C001EC
:105FC00080018001800183018301C701FF007E0001
:105FD000000000000000000000000000C000E00021
:105FE000E000F000D000D800D800CC00CC00C60003
:105FF000C600C300C300FF01FF01C000C000C00015
:10600000C000C00000000000000000000000000010
:10601000FE01FE0106000600060003007B00FF00F3
:10602000C70183018001800180018001800183011B
:106030008301C701FE007C0000000000000000009A
:1060400000000000F800FC018E01060006000300BD
:106050007B00FF00CF01870183018301830183015E
:10606000830183018601CE01FC007800000000005E
:106070000000000000000000FF01FF01800180011E
:106080008001C000C000600060006000300030008F
:106090001800180018000C000C000C000600060088
:1060A0000000000000000000000000007C00FE0076
:1060B000C600C701830183018301C701C6007C00BC
:1060C0007C00C600C701830183018301C701C600AC
:1060D000FE007C0000000000000000000000000046
:1060E00038007C00EE00C600830183018301830138
:1060F00083018301C701EE01FC01B8018001800129
:10610000C001E2007F003C00000000000000000031
:10611000000000000000000000000E001F001F0033
:106120000E00000000000000000000000000000061
:106130000E001F001F000E00000000000000000005
:1061400000000000000000000000000000001C0033
:106150003E003E001C0000000000000000000000A7
:10616000000000003C003C001C001C000E000E0063
:106170000600070000000000000000000000000012
:106180000000000080018001F0017C000F0003008E
:106190000F007C00F0018001800100000000000081
:1061A00000000000000000000000000000000000EF
:1061B0000000000000000000FF01FF0100000000DF
:1061C00000000000FF01FF010000000000000000CF
:1061D00000000000000000000000000000000000BF
:1061E00000000000000000000000000001000300AB
:1061F0001F007C00E0018001E0017C001F00030023
:10620000010000000000000000000000000000008D
:106210000000000000007C00FE00C7018201800138
:1062200080018001C00060003000180018001800D4
:10623000180000000000000038007C007C003800DE
:1062400000000000000000000000F800FC01CC018C
:10625000860186018301C301E301E301B301B301B8
:10626000B301B301B301E301C300060006000E0051
:10627000FC00F00100000000000000000000000031
:106280003800380038006C006C006C00C600C60096
:10629000C600C60083018301FF01FF018301830162
:1062A00083018301830183010000000000000000DE
:1062B000000000007F00FF00C30183018301830110
:1062C00083018301C300FF00FF00C3018301830139
:1062D000830183018301C301FF007F0000000000F0
:1062E00000000000000000007800FC00CE018601E4
:1062F0008701830103000300030003000300030080
:1063000003000300830187018601CE01FC007800B1
:106310000000000000000000000000007F00FF00FF
:10632000C30183018301830183018301830183010D
:106330008301830183018301830183018301C301FD
:10634000FF007F00000000000000000000000000CF
:10635000FF01FF010300030003000300030003002B
:106360000300FF00FF00030003000300030003001D
:1063700003000300FF01FF01000000000000000017
:1063800000000000FF01FF01030003000300030001
:10639000030003000300FF00FF00030003000300ED
:1063A00003000300030003000300030000000000DB
:1063B00000000000000000007C00FE00C701830117
:1063C000830103000300030003000300E300E30173
:1063D00083018301830183018301C701FE007C00E7
:1063E00000000000000000000000000083018301A5
:1063F0008301830183018301830183018301FF0101
:10640000FF018301830183018301830183018301F0
:106410008301830100000000000000000000000074
:10642000FF00FF00180018001800180018001800DE
:10643000180018001800180018001800180018009C
:1064400018001800FF00FF0000000000000000001E
:1064500000000000E001E001800180018001800176
:10646000800180018001800180018001830183011E
:10647000830183018301C701FE007C00000000004E
:1064800000000000000000008301830183018301FC
:10649000C3006300730033001B000F001B003B00B0
:1064A00073006300C300C30183018301830183017F
:1064B00000000000000000000000000003000300D6
:1064C00003000300030003000300030003000300B4
:1064D00003000300030003000300030003000300A4
:1064E000FF01FF01000000000000000000000000AC
:1064F000C300C300C300E700E700E700FF00FF00A0
:10650000FF00DB00DB00DB00C300C300C300C300EF
:10651000C300C300C300C30000000000000000006F
:106520000000000083018301870187018F018F0133
:106530009B019B01B301B301E301E301C301C3016B
:106540008301830183018301830183010000000033
:10655000000000000000000038007C00EE00C600D3
:10656000C7018301830183018301830183018301C7
:10657000830183018301C701C600EE007C0038005F
:106580000000000000000000000000007F00FF008D
:10659000C301830183018301830183018301C3015B
:1065A000FF007F000300030003000300030003005B
:1065B00003000300000000000000000000000000D5
:1065C00038007C00EE00C600C7018301830183010F
:1065D0008301830183018301830183018301C70157
:1065E000C600EE007C00F801800180010000000080
:1065F000000000007F00FF00C301830183018301CD
:10660000830183018301C301FF007F006300C30096
:10661000C301830183018301830183010000000022
:1066200000000000000000007C00FE00C7018300A5
:106630000300030007000E001C007800F000C001FA
:1066400080018001800180018101C301FF007E0083
:10665000000000000000000000000000FF00FF003C
:10666000180018001800180018001800180018006A
:10667000180018001800180018001800180018005A
:1066800018001800000000000000000000000000DA
:1066900083018301830183018301830183018301DA
:1066A0008301830183018301830183018301C70186
:1066B000C600EE007C003800000000000000000072
:1066C00000000000C300C300C300C300C300C30038
:1066D000C300C300C300C300660066006600660016
:1066E0003C003C003C0018001800180000000000AE
:1066F0000000000000000000C300C300C300C3008E
:10670000C300DB00DB00DB00DB00DB00DB00DB00C9
:10671000DB00FF00E700E700E700C300C300C300A1
:10672000000000000000000000000000C300C300E3
:10673000C300660066003C0018001800180018002E
:1067400018003C003C0066006600C300C300C300A4
:10675000C300C300000000000000000000000000B3
:10676000C300C300C300C300C300C30066006600CB
:1067700024003C003C001800180018001800180005
:1067800018001800180018000000000000000000A9
:1067900000000000FF01FF018001C000C000600098
:1067A000600070003000180018001C000C0006008B
:1067B0000600070003000300FF01FF0100000000C6
:1067C0000000000000000000FF00FF0003000300C5
:1067D00003000300030003000300030003000300A1
:1067E000030003000300030003000300FF00FF0099
:1067F0000000000000000000000000000300030093
:10680000030003000300060006000C000C000C004F
:10681000180018003000300060006000C000C000A8
:10682000C000C000000000000000000000000000E8
:10683000FF00FF00C000C000C000C000C000C000DA
:10684000C000C000C000C000C000C000C000C00048
:10685000C000C000FF00FF000000000000000000BA
:1068600000000000180018003C006600C300C300D0
:10687000C300000000000000000000000000000055
:106880000000000000000000000000000000000008
:1068900000000000000000000000000000000000F8
:1068A00000000000000000000000000000000000E8
:1068B00000000000000000000000000000000000D8
:1068C000FF03FF03000000000000000006001F009F
:1068D0007C00E0000000000000000000000000005C
:1068E00000000000000000000000000000000000A8
:1068F0000000000000000000000000000000000098
:10690000000000000000000000007E00FF00C20147
:1069100080018001BC01FE01C70183018301830165
:106920008301C7017E01BC010000000000000000DF
:1069300000000000030003000300030003003B000D
:106940007F00E700C300830183018301830183018A
:1069500083018301C300E7007D00390000000000CF
:106960000000000000000000000000000000000027
:1069700000007C00FE00C701830103010300030047
:1069800003000300030003008301C701FE007C0035
:1069900000000000000000000000000080018001F5
:1069A000800180018001B801FC01CE0186018301D4
:1069B00083018301830183018301830186018E01A9
:1069C000FC01380100000000000000000000000091
:1069D000000000000000000000003C007E00E70016
:1069E000C3018301C301FF007F0003000300030014
:1069F00003008701FE01FC00000000000000000011
:106A000000000000F000F8011C010C000C000C005C
:106A10003F003F000C000C000C000C000C000C00B0
:106A20000C000C000C000C000C000C00000000001E
:106A3000000000000000000000009C01BE01E70112
:106A40008301830183018301830183018301830126
:106A50008301E701BE019C0180018001C001C200E9
:106A6000FF003C00000000000000000003000300E5
:106A70000300030003007300FB00CF018F018701B7
:106A800083018301830183018301830183018301E6
:106A900083018301000000000000000000000000EE
:106AA000380038000000000000003F003F003000C8
:106AB0003000300030003000300030003000300056
:106AC0003000300030003000000000000000000006
:106AD00000000000600060000000F801F801800183
:106AE000800180018001800180018001800180019E
:106AF0008001800183018301C301C600FE007C0088
:106B00000000000000000000030003000300030079
:106B10000300830183018301C301C30063003300C9
:106B20003F0077006300C300830183018301830179
:106B30000000000000000000000000003F003F00D7
:106B400030003000300030003000300030003000C5
:106B500030003000300030003000300030003000B5
:106B600030003000000000000000000000000000C5
:106B700000000000000000000000B601BE01F601A8
:106B8000B601B601B601B601B601B601B601B6014D
:106B9000B601B601B601B601000000000000000019
:106BA0000000000000000000000000000000630082
:106BB000F700F6019E018E0186018601860186019D
:106BC000860186018601860186018601000000009B
:106BD00000000000000000000000000000000000B5
:106BE000000038007C00EE00C600830183018301B1
:106BF0008301830183018301C600EE007C0038001D
:106C00000000000000000000000000000000000084
:106C10006300F700DE018601860186018601860198
:106C20008601860186018E01DE01F60066000600FF
:106C3000060006000600060000000000000000003C
:106C4000000000009C01BE01F700E300C300C30088
:106C5000C300C300C300C300C300E300F700FE008D
:106C6000DC00C000C000C000C000C0000000000088
:106C700000000000000000000000000000006300B1
:106C8000F3009B018E018E0106000600060006003F
:106C900006000600060006000600060000000000D0
:106CA00000000000000000000000000000000000E4
:106CB00000007C00FE0043000300030003001F00EF
:106CC0007E00F000C000C000C000C3007F003E0096
:106CD00000000000000000000000000000000C00A8
:106CE0000C000C000C00FF00FF000C000C000C005E
:106CF0000C000C000C000C000C000C008C019C0122
:106D0000F801F0000000000000000000000000009A
:106D100000000000000000000000830183018301E7
:106D20008301830183018301830183018301C30103
:106D3000E301A701BE019C0100000000000000006B
:106D400000000000000000000000000000008301BF
:106D50008301830183018301C600C600C600C6000B
:106D60006C006C006C002800380038000000000047
:106D70000000000000000000000000000000000013
:106D80000000C300C300C300DB00DB00DB00DB004E
:106D9000DB00FF00FF00E700E700C300C300C30003
:106DA00000000000000000000000000000000000E3
:106DB000000000000000C300C300660066003C0045
:106DC0003C00180018003C003C0066006600C30050
:106DD000C300C3000000000000000000000000002D
:106DE0000000000083018301830183018301860188
:106DF0008601C600CC006C006C006C0038003000CE
:106E000030003000300019001F00070000000000B3
:106E10000000000000000000000000000000FF0172
:106E2000FF018001C000E000600030003800180061
:106E30000C000E0006000300FF01FF01000000002F
:106E40000000000000000000E00070003000300092
:106E50003000300030003000300018000F000F000C
:106E600018003000300030003000300030003000BA
:106E70007000E000000000000000000003000300BC
:106E800003000300030003000300030003000300EA
:106E900003000300030003000300030003000300DA
:106EA00003000300030003000000000000000000D6
:106EB0000E001C0018001800180018001800180018
:106EC0003000E001E0013800180018001800180038
:106ED00018001800180018001C000E000000000028
:106EE000000000001C033F03E303C3010000000097
:106EF0000000000000000000000000000000000092
:106F00000000000000000000000000000000000081
:106F10000000000000000000000000000000000071
:106F20000000000000000000000000000000000061
:106F30000000000000000000000000000000000051
:106F40000000000000000000000000001800180011
:106F500018003C003C003C006600660066006600CD
:106F6000C300C300FF00FF00C300C300C300C30091
:106F7000C300C3000000000000000000000000008B
:106F8000FF01FF018301030003000300030003006E
:106F90007F00FF00C301830183018301830183011B
:106FA0008301C301FF007F0000000000000000001B
:106FB000000000007F00FF00C30183018301830103
:106FC00083018301C300FF00FF00C301830183012C
:106FD000830183018301C301FF007F0000000000E3
:106FE0000000000000000000FF01FF018301030119
:106FF0000300030003000300030003000300030079
:107000000300030003000300030003000300030068
:10701000000000000000000000000000C001E001CE
:10702000B001B001B001B8019801980198019C012C
:107030008C018C018C018E018601860186018601FE
:10704000FE01FE0103030303000000000000000036
:10705000FF01FF010300030003000300030003001E
:107060000300FF00FF000300030003000300030010
:1070700003000300FF01FF0100000000000000000A
:1070800000000000DB00DB00DB00DB00DB00DB00DE
:10709000DB00DB007E003C003C007E00DB00DB0010
:1070A000DB00DB00DB00DB00DB00DB0000000000BE
:1070B00000000000000000001C007E00E300C30090
:1070C000C000C000C000C00060003C007E00C000E6
:1070D00080018001800180018301C701FE007C00E6
:1070E0000000000000000000000000008301830198
:1070F0008301C301C301E301B301B3019B019B0100
:107100009B019B019B018F018F01870183018301FB
:107110008301830100000000000000000000000067
:107120003800BB018301C301C301E301E301B301E3
:10713000B3019B019B019B019B018F018F01870183
:10714000830183018301830100000000000000002F
:107150000000000083018301C300C30063006300DB
:10716000330033003F003F0073006300E300C301BE
:1071700083018301830183018301830100000000F7
:107180000000000000000000F001FC018C018E01F5
:1071900086018601860187018301830183018301C2
:1071A00083018301830183018301830183018301BF
:1071B000000000000000000000000000C300C30049
:1071C000C300E700E700FF00FF00DB00DB00DB009F
:1071D000DB00DB00C300C300C300C300C300C30067
:1071E000C300C30000000000000000000000000019
:1071F000830183018301830183018301830183016F
:107200008301FF01FF018301830183018301830166
:10721000830183018301830100000000000000005E
:107220000000000038007C00EE00C600C7018301AA
:10723000830183018301830183018301830183012E
:107240008301C701C600EE007C003800000000008A
:107250000000000000000000FF01FF018301830126
:1072600083018301830183018301830183018301FE
:1072700083018301830183018301830183018301EE
:107280000000000000000000000000007F00FF0080
:10729000C301830183018301830183018301C3014E
:1072A000FF007F000300030003000300030003004E
:1072B00003000300000000000000000000000000C8
:1072C0007800FC00CE0186018701830103000300E2
:1072D0000300030003000300030003008301870190
:1072E0008601CE01FC0078000000000000000000D4
:1072F00000000000FF00FF00180018001800180030
:1073000018001800180018001800180018001800BD
:1073100018001800180018001800180000000000DD
:10732000000000000000000083018301830183014D
:10733000830183018301830183018701FE01F80139
:1073400080018001800181018301C701FE007C0072
:107350000000000000000000000000003C007E0073
:10736000DB00DB00DB00DB00DB00DB00DB00DB0045
:10737000DB007E003C001800180018001800180000
:1073800018001800000000000000000000000000CD
:10739000C300C300C300C300C300C300660066008F
:1073A0003C00180018003C0066006600C300C300E3
:1073B000C300C300C300C3000000000000000000C1
:1073C000000000006300630063006300630063006B
:1073D0006300630063006300630063006300630095
:1073E0006300630063006300FF01FF018001800010
:1073F000000000000000000083018301830183017D
:107400008301830183018301830183018701FE01DD
:10741000F8018001800180018001800180018001EC
:10742000000000000000000000000000C300C300D6
:10743000DB00DB00DB00DB00DB00DB00DB00DB0074
:10744000DB00DB00DB00DB00DB00DB00DB00DB0064
:10745000FF00FF000000000000000000000000002E
:10746000C300C300DB00DB00DB00DB00DB00DB0074
:10747000DB00DB00DB00DB00DB00DB00DB00DB0034
:10748000DB00DB00FF00FF00C000C00000000000C8
:1074900000000000030003000300030003000300DA
:1074A000030003007F00FF00C30183018301830108
:1074B000830183018301C301FF007F0000000000FE
:1074C00000000000000000008301830183018301AC
:1074D00083018301830183019F01BF01B301B301D4
:1074E000B301B301B301B301B301B301BF019F0104
:1074F0000000000000000000000000000F000F006E
:107500000D000C000C000C000C000C007C00FC00BA
:10751000DC018C018C018C018C018C018C01DC0163
:10752000F8007000000000000000000000000000F3
:107530007C00FE00C701830183018301800180017B
:107540008001F801F801800180018001830183013D
:107550008301C701FE007C00000000000000000065
:1075600000000000E300E301B301B301B3019B019C
:107570009B019B019B019F019F019B019B019B0123
:107580009B01B301B301B301E301E300000000007C
:107590000000000000000000F801FE0187018301E7
:1075A000830183018301830186019E01FC01F001B7
:1075B000B80198019C018C01860187018301830138
:1075C00000000000000000000000000000000000BB
:1075D0000000000000007E00FF00C2018001800169
:1075E000BC01FE01C7018301830183018301C7013F
:1075F0007E013C0100000000000000000000860148
:10760000CF01FB0003000E001C007000FC00CE0147
:107610008601830183018301830183018301830147
:107620008701CE01FC00780000000000000000008F
:1076300000003C007E00630033001B000F00770059
:10764000FB00C7018701830183018301830183015B
:10765000830183018601CE01FC0078000000000058
:10766000000000000000000000000000000000001A
:1076700000007E00FF00C201800180018001F00156
:10768000FC001E000700030003008701FE01FC0050
:107690000000000000000000000000003C00F800B6
:1076A000C00180018001B801FC01CE018601830187
:1076B0008301830183018301830183018601CE015C
:1076C000FC00780000000000000000000000000046
:1076D000000000000000000000007800FC00CE0167
:1076E00086018301C301FF007F0003000300030044
:1076F00006008E01FC01F8010000000000000000FF
:107700000000000000000000000000000000DB009E
:10771000DB00DB007E003C0018003C007E00DB004C
:10772000DB00DB00DB00DB00DB00DB000000000037
:107730000000000000000000000000000000000049
:1077400000003C007E00E700C300C30060003C0076
:107750007C00C00080018001C301E7007E003C0086
:107760000000000000000000000000000000000019
:107770000000000000008301830183018301830175
:1077800083018301830183018301C301C301A70135
:10779000BE019C010000000000000000000000008D
:1077A0000000000000003C001800830183018301F9
:1077B0008301830183018301830183018301C30169
:1077C000E301A701BE019C010000000000000000D1
:1077D0000000000000000000000000000000830125
:1077E0008301C3006300630033001B003F00770088
:1077F0006300C30083018301830183010000000053
:107800000000000000000000000000000000000078
:107810000000F001F8018C018C018C018C018601C3
:10782000860186018601830183018301830183012F
:107830000000000000000000000000000000000048
:107840000000000000008100C300E700FF00FF000F
:10785000DB00DB00DB00DB00C300C300C300C300B0
:10786000C300C30000000000000000000000000092
:10787000000000000000000000008301830183017C
:10788000830183018301FF01FF01830183018301E0
:1078900083018301830183010000000000000000D8
:1078A00000000000000000000000000000003800A0
:1078B0007C00EE00C6008301830183018301830104
:1078C00083018301C600EE007C0038000000000048
:1078D00000000000000000000000000000000000A8
:1078E0000000FF01FF018301830183018301830104
:1078F0008301830183018301830183018301830168
:107900000000000000000F0F0F0F0F0F0F0F0F0FE1
:10791000000000000000000000000F0F0F0F0F0F0D
:107920000F0F0F0F000000000000000000000F0FFD
:107930000F0F0F0F0F0F0F0F00000F0F0F0F0F0F75
:107940000F0F0F0FF0F0F0F0F0F0F0F0F0F00F0F7D
:107950000F0F0F0F0F0F0F0FF0F0F0F0F0F0F0F02F
:10796000F0F00F0F0F0F0F0F0F0F0F0F0000FFFFA3
:10797000FFFFFFFFFFFF0F0F0F0F0F0F0F0F0F0F77
:107980000F0FFFFFFFFFFFFFFFFF0F0F0F0F0F0F87
:107990000F0F0F0F0F0FFFFFFFFFFFFFFFFF0F0F77
:1079A0000000800180018001800180018001800150
:1079B00080018001800180018001800180018001BF
:1079C00080018001800180018001800180018001AF
:1079D0008001800100008001800180018001800120
:1079E000800180018001800180018001800180018F
:1079F0008001FF01FF018001800180018001800181
:107A000080018001800180010000800180018001EF
:107A1000800180018001800180018001800180015E
:107A2000FF01FF01800180018001FF01FF01800152
:107A3000800180018001800180018001000030060A
:107A40003006300630063006300630063006300686
:107A5000300630063006300630063F063F06300658
:107A60003006300630063006300630063006300666
:107A70000000000000000000000000000000000006
:107A80000000000000000000000000000000FF07F0
:107A9000FF07300630063006300630063006300666
:107AA000300630060000000000000000000000006A
:107AB000000000000000000000000000FF01FF01C6
:107AC000800180018001FF01FF01800180018001B0
:107AD0008001800180018001000030063006300600
:107AE00030063006300630063006300630063006E6
:107AF0003F063F060006000600063F063F0630062A
:107B000030063006300630063006300600003006FB
:107B100030063006300630063006300630063006B5
:107B200030063006300630063006300630063006A5
:107B30003006300630063006300630063006300695
:107B40000000000000000000000000000000000035
:107B50000000000000000000FF07FF07000600060D
:107B600000063F063F063006300630063006300677
:107B7000300630060000300630063006300630068B
:107B80003006300630063006300630063F063F0627
:107B9000000600060006FF07FF07000000000000C7
:107BA0000000000000000000000030063006300633
:107BB0003006300630063006300630063006300615
:107BC000300630063006FF07FF0700000000000007
:107BD0000000000000000000000000000000800124
:107BE000800180018001800180018001800180018D
:107BF00080018001FF01FF01800180018001FF0100
:107C0000FF01000000000000000000000000000074
:107C10000000000000000000000000000000000064
:107C2000000000000000000000000000FF01FF0154
:107C3000800180018001800180018001800180013C
:107C400080018001000080018001800180018001AD
:107C5000800180018001800180018001800180011C
:107C6000800180FF80FF0000000000000000000095
:107C70000000000000000000000080018001800181
:107C800080018001800180018001800180018001EC
:107C9000800180018001FFFFFFFF00000000000065
:107CA00000000000000000000000000000000000D4
:107CB00000000000000000000000000000000000C4
:107CC00000000000000000000000FFFFFFFF800137
:107CD000800180018001800180018001800180019C
:107CE000000080018001800180018001800180010D
:107CF000800180018001800180018001800180FF7E
:107D000080FF80018001800180018001800180016D
:107D10008001800100000000000000000000000061
:107D20000000000000000000000000000000000053
:107D30000000FFFFFFFF0000000000000000000047
:107D400000000000000000000000800180018001B0
:107D5000800180018001800180018001800180011B
:107D6000800180018001FFFFFFFF80018001800111
:107D7000800180018001800180018001000080017C
:107D800080018001800180018001800180018001EB
:107D90008001800180FF80FF80018001800180FFE1
:107DA00080FF8001800180018001800180018001CD
:107DB0000000300630063006300630063006300649
:107DC000300630063006300630063006300630FE0B
:107DD00030FE3006300630063006300630063006FB
:107DE0003006300600003006300630063006300619
:107DF00030063006300630063006300630FE30FEE3
:107E0000300030003000F0FFF0FF00000000000004
:107E10000000000000000000000000000000000062
:107E20000000000000000000000000000000000052
:107E3000F0FFF0FF30003000300030FE30FE300642
:107E400030063006300630063006300600003006B8
:107E50003006300630063006300630063006300672
:107E6000300630063FFE3FFE000000000000FFFF2E
:107E7000FFFF000000000000000000000000000004
:107E800000000000000000000000000000000000F2
:107E90000000000000000000FFFFFFFF00000000E6
:107EA00000003FFE3FFE300630063006300630064A
:107EB0003006300600003006300630063006300648
:107EC00030063006300630063006300630FE30FE12
:107ED00030003000300030FE30FE30063006300614
:107EE00030063006300630060000000000000000BA
:107EF0000000000000000000000000000000000082
:107F0000FFFFFFFF000000000000FFFFFFFF000079
:107F1000000000000000000000000000000030062B
:107F200030063006300630063006300630063006A1
:107F3000300630063FFE3FFE0000000000003FFE1E
:107F40003FFE30063006300630063006300630067A
:107F5000000080018001800180018001800180019A
:107F60008001800180018001FFFFFFFF0000000011
:107F70000000FFFFFFFF0000000000000000000005
:107F800000000000000030063006300630063006E3
:107F90003006300630063006300630063006300631
:107FA0003006FFFFFFFF000000000000000000009F
:107FB00000000000000000000000000000000000C1
:107FC00000000000000000000000000000000000B1
:107FD000FFFFFFFF000000000000FFFFFFFF800128
:107FE000800180018001800180018001000000008B
:107FF0000000000000000000000000000000000081
:1080000000000000000000000000FFFFFFFF30063E
:1080100030063006300630063006300630063006B0
:1080200000003006300630063006300630063006D6
:108030003006300630063006300630063006F0FFD7
:10804000F0FF000000000000000000000000000041
:10805000000000000000800180018001800180019B
:1080600080018001800180018001800180FF80FF0C
:1080700080018001800180FF80FF0000000000007F
:1080800000000000000000000000000000000000F0
:1080900000000000000000000000000000000000E0
:1080A00080FF80FF80018001800180FF80FF8001D0
:1080B00080018001800180018001800100000000BA
:1080C00000000000000000000000000000000000B0
:1080D00000000000000000000000F0FFF0FF30068C
:1080E00030063006300630063006300630063006E0
:1080F0000000300630063006300630063006300606
:108100003006300630063006300630063006FFFFF7
:10811000FFFF3006300630063006300630063006E7
:10812000300630060000800180018001800180015E
:10813000800180018001800180018001FFFFFFFF3D
:10814000800180018001FFFFFFFF8001800180012D
:108150008001800180018001000080018001800198
:108160008001800180018001800180018001800107
:10817000800180018001FF01FF010000000000007C
:1081800000000000000000000000000000000000EF
:1081900000000000000000000000000000000000DF
:1081A000000000000000000080FF80FF80018001CF
:1081B00080018001800180018001800180018001B7
:1081C0000000FFFFFFFFFFFFFFFFFFFFFFFFFFFFBD
:1081D000FFFFFFFFFFFFFFFFFFFFFFFFFFFFFFFFAF
:1081E000FFFFFFFFFFFFFFFFFFFFFFFFFFFFFFFF9F
:1081F000FFFFFFFF00000000000000000000000083
:10820000000000000000000000000000000000006E
:1082100000000000FFFFFFFFFFFFFFFFFFFFFFFF6A
:10822000FFFFFFFFFFFFFFFF0000FF00FF00FF0059
:10823000FF00FF00FF00FF00FF00FF00FF00FF0046
:10824000FF00FF00FF00FF00FF00FF00FF00FF0036
:10825000FF00FF00FF00FF00FF00FF000000E00341
:10826000E003E003E003E003E003E003E003E003F6
:10827000E003E003E003E003E003E003E003E003E6
:10828000E003E003E003E003E003E003E003E003D6
:1082900000000000000000000000000000000000DE
:1082A00000000000000000000000000000000000CE
:1082B000FF03FF03FF03FF03FF03FF03FF03FF03AE
:1082C000FF03FF03000000000000000000000000AA
:1082D00000007300FB00CF0187018301830183014C
:1082E00083018301830183018301C701FF007B00B8
:1082F0000300030003000300000000000000000072
:10830000000000000000000000007800FC00CE012A
:1083100086010300030003000300030003000300C1
:108320008601CE01FC007800000000000000000083
:108330000000000000000000000000000000FF003E
:10834000FF00DB00DB001800180018001800180000
:10835000180018001800180018001800000000008D
:10836000000000000000000000000000000000000D
:108370000000830183018301830183018301830161
:108380008701FE01FC0180018101C301FE007C0028
:1083900000000000000000000000000000000000DD
:1083A00000000000000018003C007E00DB00DB0045
:1083B000DB00DB00DB00DB007E003C001800180067
:1083C000180018000000000000000000000000007D
:1083D0000000000000000000000083018301C701CD
:1083E000C6006C006C00380038006C006C00C600E1
:1083F000C701830183018301000000000000000029
:1084000000000000000000000000000000008301E8
:10841000830183018301830183018301830183013C
:108420008301830183018701FE01780180018001BE
:10843000000000000000000000000000000000003C
:108440000000830183018301830183018301830190
:108450008701FE01F8018001800180018001800117
:10846000000000000000000000000000000000000C
:10847000000000000000DB00DB00DB00DB00DB00B5
:10848000DB00DB00DB00DB00DB00DB00DB00DB0014
:10849000FF00FF00000000000000000000000000DE
:1084A000000000000000000000000000DB00DB0016
:1084B000DB00DB00DB00DB00DB00DB00DB00DB00E4
:1084C000DB00DB00FF00FF008001800100000000F6
:1084D0000000000000000000000000000000070095
:1084E00007000600060006000600E600F6019E01F1
:1084F0008E0186018601C601FE007C00000000009E
:10850000000000000000000000000000000000006B
:1085100000008301830183018301830183019B01A7
:10852000BF01BF01B301B301B301B301BF019F019B
:10853000000000000000000000000000000000003B
:10854000000000000000030003000300030003001C
:1085500003007B00FF008701830183018301C301C6
:10856000FF007F000000000000000000000000008D
:10857000000000000000000000007C00FE00C701B9
:10858000830181018001C801FC01B80180018001E3
:108590008301C701FE007C00000000000000000015
:1085A0000000000000000000000000000000630068
:1085B0006300F300F3009B019B019F019F019B015E
:1085C0009B019B01F300F3006300630000000000C7
:1085D000000000000000000000000000000000009B
:1085E0000000F801FC0186018301830183018701FA
:1085F000FE01F801E001B00198018C0186018301C0
:108600000000000000000000000000009801980138
:108610000000FF01FF010300030003000300FF004F
:10862000FF00030003000300030003000300030036
:10863000FF01FF010000000000000000000000003A
:1086400000000000CC00CC0000007C00FE00C70150
:10865000830183018301C301FF007F000300030046
:1086600083018701FE01FC00000000000000000003
:1086700000000000000000000000000000000000FA
:10868000000000000000000000008000C00060004A
:10869000300018000C00060003000100000000007C
:1086A00000000000000000000000000000000000CA
:1086B00000000000000000000000000001000300B6
:1086C00006000C00180030006000C00080010001AE
:1086D0000000000000000000000000000001800118
:1086E000C0006000300018000C000600030001000C
:1086F000000000000000000000000000000000007A
:108700000000000000000000000000000000000069
:108710000100030006000C00180030006000C000DB
:1087200080010001000000000000000000000000C7
:108730000000000000000000000000000000000039
:1087400000000000000000000000000000003000F9
:108750006000C000FF01FF01C000300030000000D9
:108760000000000000000000000000000000000009
:1087700000000000000000000000000000000000F9
:10878000000018000C000600FF01FF0106000C00AD
:1087900018000000000000000000000000000000C1
:1087A00000000000000000000000000000000000C9
:1087B0000000000000000000180018001800180059
:1087C000180018009900DB007E003C001800000033
:1087D0000000000000000000000000000000000099
:1087E00000000000000000000000000018003C0035
:1087F0007E00DB009900180018001800180018000F
:108800001800000000000000000000000000000050
:108810000000000000000000000000001800180028
:1088200000000000FF00FF0000000000180018001A
:108830000000000000000000000000000000000038
:1088400000000000000000000000180018001800E0
:1088500018001800FF00FF0018001800180018008A
:108860001800000000000000FF00FF0000000000F2
:10887000000000000000000000000000C302C3026E
:10888000C302C702C702C700CF00CF00DB00DB0076
:10889000DB00F300F300E300E300C300C300C30008
:1088A000C300C30000000000000000000000000042
:1088B000000000000000000001033903FE00C701B2
:1088C0008301830183018301C701FE003901010196
:1088D0000000000000000000000000000000000098
:1088E0000000000000000000000000000000000088
:1088F000000000007F007F007F00000000000000FB
:108900000000000000000000000000000000000067
:02891000000065
:00000001FF
